:0200000480007A
:10000000B72F0000938F0F8073900F3015A8130047
:100010000000130000001300000013000000130094
:100020000000130000001300000013000000130084
:100030000000130000001300000013000000010086
:10004000970200009382020C73905230814001416C
:100050008141014281420143814301448144014580
:100060008145014681460147814701488148014950
:100070008149014A814A014B814B014C814C014D20
:10008000814D014E814E014F814F971102009381A6
:10009000E1E1170502001305E56297A503009385CA
:1000A000A58301461122170502001305E5539705A4
:1000B00002009385655F0146C52817B50300130547
:1000C000E58197C503009385258137B6ABAB130651
:1000D000B6BAD92817C1030013014180EF60304937
:1000E000860293D21200F512638802008242110147
:1000F0006F00001073002030824211017300203025
:10010000711116C0F3222034E3CC02FC82421101AB
:10011000130141F806C20AC40EC612C816CA1ACC88
:100120001ECE22D026D22AD42ED632D836DA3ADCC7
:100130003EDEC2C0C6C2CAC4CEC6D2C8D6CADACC97
:10014000DECEE2D0E6D2EAD4EED6F2D8F6DAFADCA7
:10015000FEDE73252034F32510340A8601A07310C7
:10016000153492402241B2414242D2426243F243AC
:10017000025492542255B2554256D2566257F25703
:10018000064896482649B649464AD64A664BF64B33
:10019000065C965C265DB65D465ED65E665FF65F83
:1001A0001301C1077300203010C16374B50011053D
:1001B000E5BF828000000000000000000000000099
:1001C000000000000000000000000000000000002F
:1001D000000000000000000000000000000000001F
:1001E000000000000000000000000000000000000F
:1001F000197106C00AC20EC412C616C81ACA1ECC8D
:1002000022CE26D02AD22ED432D636D83ADA3EDCC6
:1002100042DEC6C0CAC2CEC4D2C6D6C8DACADECC96
:10022000E2CEE6D0EAD2EED4F2D6F6D8FADAFEDCA6
:100230009702020083A2823E23A02200F322103400
:1002400096DEEF00002B170102000321213D024141
:10025000F65273901234B72200009382028873A082
:10026000023082403242C2425243E24372448254DC
:100270001255A2553256C2565257E2577258864806
:100280001649A649364AC64A564BE64B764C865C1A
:10029000165DA65D365EC65E565FE65F0961730059
:1002A0002030970202009382E24123A0120023A291
:1002B000220023A4320023A6420023A8520023AA2E
:1002C000620023AC720023AE820023A0920223A21C
:1002D000A20223A4B20223A6C20223A8D20223AA06
:1002E000E20223ACF20223AE020323A0120523A2F2
:1002F000220523A4320523A6420523A8520523AADA
:10030000620523AC720523AE820523A0920723A2C7
:10031000A20723A4B20723A6C20723A8D20723AAB1
:10032000E20723ACF207EF4050301701020003212F
:10033000E12E0241F65273901234B72200009382EC
:10034000028873A0023082403242C2425243E243EA
:10035000724482541255A2553256C2565257E25731
:10036000725886481649A649364AC64A564BE64B45
:10037000764C865C165DA65D365EC65E565FE65FB1
:10038000096173002030970202009382A23383A098
:10039000020003A1420083A1820003A2C20083A243
:1003A000020103A3420183A3820103A4C20183A427
:1003B000020203A5420283A5820203A6C20283A60B
:1003C000020303A7420383A7820303A8C20383A8EF
:1003D000020403A9420483A9820403AAC20483AAD3
:1003E000020503AB420583AB820503ACC20583ACB7
:1003F000020603AD420683AD820603AEC20683AE9B
:10040000020703AFC20983AF820782807370043092
:10041000197106C00AC20EC412C616C81ACA1ECC6A
:1004200022CE26D02AD22ED432D636D83ADA3EDCA4
:1004300042DEC6C0CAC2CEC4D2C6D6C8DACADECC74
:10044000E2CEE6D0EAD2EED4F2D6F6D8FADAFEDC84
:100450009702020083A2821C23A0220086DEEF20E6
:100460004037170102000321611B0241F6527390CD
:100470001234B72200009382028873A002308240B7
:100480003242C2425243E243724482541255A25550
:100490003256C2565257E257725886481649A649F4
:1004A000364AC64A564BE64B764C865C165DA65DD0
:1004B000365EC65E565FE65F09617300203073707A
:1004C000043001A07310453082807325403073F0F2
:1004D00043308280970700009387A7FE232EB5FE46
:1004E0002322C5FA232635F82320F5F8130505F84D
:1004F0008280411106C6EF407010EF10301501E503
:10050000B24041018280B24041016F20802C9307AC
:1005100085007D575CC118C55CC51CC9232005003A
:1005200082802328050082805C41DCC1984798C501
:1005300098474CC38CC788C91C4185071CC1828061
:100540009041FD57130785006314F60039A83E87D4
:100550005C439443E37DD6FEDCC18CC798C54CC395
:1005600088C91C4185071CC1828018495C43EDB7CE
:10057000584114451C4914C71845544154C3D84325
:100580006314A7001845D8C32328050088437D15A8
:1005900088C382803041AE8701CE4C455841B29528
:1005A0004CC563E4E5000C414CC53E856F30902995
:1005B0008280411122C406C62A8426C2EF20101B65
:1005C0003C44635BF0025C5085CB9304440209A871
:1005D0003C44FD173CC43C446350F0025C5089CF5E
:1005E0002685EF2020616DD5EF2010013C44FD17DA
:1005F0003CC43C44E344F0FEFD573CC4EF2050199A
:10060000EF20D0167C40635BF0021C4885CB93043E
:10061000040109A87C40FD177CC07C406350F002B7
:100620001C4889CF2685EF20E05C6DD5EF20C07C8B
:100630007C40FD177CC07C40E344F0FEFD577CC04D
:100640002244B240924441016F20901429CD0111FF
:1006500022CC2A8406CE26CA4AC84EC62E89EF204E
:10066000F01024404C5C832904002685EF60C059BB
:100670007D57232C0402B3079540CE974E9578C042
:1006800048C0232434015CC438C4631109021C48E7
:100690008DE7EF20F00FF2406244D2444249B24964
:1006A0000545056182807370043001A013050401C3
:1006B000B93D13054402A13DE9BF13050401EF2034
:1006C00060538547E317F5FC9133E1B701E573709B
:1006D000043001A0011126CA4AC84EC606CE22CC5B
:1006E000AA842E89B289A5C9EF6000521305550569
:1006F000EF30007D2A8435C5930745051CC144DCD5
:1007000023202405EF20900624404C5C032904009C
:100710002685EF60604FFD56232C0402B3079540F9
:100720003307A900CA9774C058C05CC434C4130509
:10073000040123242401E13B13054402C93BEF20BB
:100740003005230834052285F2406244D2444249F0
:10075000B2490561828013054005EF3060762A8436
:1007600001E57370043001A000C051BF01E5737052
:10077000043001A06375B5007370043001A041110D
:1007800022C409462E84814506C6893711C500DD7D
:10079000B2402244410182807370043001A05D7137
:1007A00086C6A2C4A6C2CAC04EDE52DC56DA5AD8E9
:1007B0005ED632C6630A051C6382051C89476399AD
:1007C000F600585D85476305F7007370043001A09B
:1007D0003689AE842A84EF20A06411E5B24781C730
:1007E0007370043001A0EF206078185C5C5C014BF2
:1007F000894BFD59130A0401930A44026365F70CFF
:1008000063077919B2476381072463150B00280831
:10081000EF206051EF20C077EF10005AEF200075F5
:100820007C4063943701232204043C4463943701E1
:1008300023240404EF20C0756C002808EF20C0506A
:10084000631E051EEF208072185C5C5C630CF70A67
:10085000EF200074EF2080713C44634FF00039A812
:100860005685EF20203919C1EF2000593C44FD176F
:100870003CC43C446354F0005C50FDF32324340535
:10088000EF200071EF20806E7C40634FF00039A8AC
:100890005285EF20203619C1EF2000567C40FD170D
:1008A0007CC07C406354F0001C48FDF323223405D7
:1008B000EF20006EEF104075054BEF20206B185CA9
:1008C0005C5CE37FF7F230406305060C631F09129E
:1008D0000844A685EF3000771C4434405840B69752
:1008E0001CC463EAE70A1C5C14405850850714C412
:1008F0001CDC5DC713054402EF20C02F8547631140
:10090000F50AC9A8EF20C068B2455285EF20401013
:10091000EF20C0653C44634FF00039A85685EF20B6
:10092000602D19C1EF20404D3C44FD173CC43C44B0
:100930006354F0005C50FDF323243405EF20406540
:10094000EF20C0627C40634FF00039A85285EF2051
:10095000602A19C1EF20404A7C40FD177CC07C40D2
:100960006354F0001C48FDF323223405EF2040625D
:10097000EF10806931F1593C054B81B73C41E38F61
:1009800007E27370043001A07370043001A030409E
:1009900021E61C4085C71C5C585085071CDC39FBD0
:1009A000EF20005F0545B640264496440649F259BB
:1009B000625AD25A425BB25B616182804840EF204A
:1009C00040521C5C58502322040085071CDCE313B2
:1009D00007F279D5253CE9B74844A685EF30806613
:1009E0003C4058441440B307F0403E9758C4637CE1
:1009F000D7025840BA975CC409475C506306E902C5
:100A0000185C050718DCC9DFF5B54844A685EF304A
:100A100060633C4058441440B307F0403E9758C4CC
:100A2000E37CD7FCF9B75C50185C79DB185C7D1768
:100A300018DC185C050718DCA5D76DBD2285953E2E
:100A4000EF10805C014585B7EF2080540145A1BFC0
:100A5000411126C2AA841305400522C406C6EF3000
:100A600020462A8415CD232C0502FD577CC105475D
:100A7000410558DC3CC42322040023200400232425
:100A80000400232604002320040423089404413492
:100A900013054402AD3C8146014681452285013360
:100AA0002285B24022449244410182800DC5411109
:100AB00022C426C206C64AC0032945002A84EF2064
:100AC00060358144630CA900B24022442685024966
:100AD0009244410182807370043001A05C448544DB
:100AE000FD175CC4F5F381460146814522854539F1
:100AF000E1BF31CDA1C9011122CC26CA4AC852C4D6
:100B000006CE4EC68947B68432892E8A2A846399D6
:100B1000F600585D8547630FF7047370043001A039
:100B20006D32185C5C5CAA896366F70281444E856D
:100B3000513AF240624426854249D244B249224A9F
:100B4000056182803C41C5DB7370043001A0737085
:100B5000043001A0304041E21C40D5CB1C5C7D57E5
:100B600085071CDC3C446387E7083C4485448507D3
:100B70003CC475BF993A185C5C5CAA89636DF70246
:100B8000304079DA4844D285EF30C04B3C4058447D
:100B90001440B307F0403E9758C46375D7005840DF
:100BA000BA975CC48947E39BF4FA1C5CC5DB1C5C08
:100BB000FD171CDC65B7304045D24844D285EF3084
:100BC00060483C4058441440B307F0403E9758C436
:100BD000E367D7FCD9BFDDF40844D285EF30804607
:100BE0001C4434405840B6971CC4E3E9E7F61C4067
:100BF0001CC4ADB75C5085449DDB13054402EF1067
:100C0000707F15D5E30509F2232099000DB7484000
:100C1000EF20202D2322040091B721CD3C4181C734
:100C20007370043001A01C41A1CB011122CC26CA53
:100C30002A844AC84EC606CE2E894138185C5C5CB0
:100C4000AA898144637DF7001C5C7D5785071CDC05
:100C50003C446388E7023C44854485073CC44E8598
:100C60009530F240624426854249D244B24905613A
:100C700082807370043001A05C41C5DB7370043066
:100C800001A05C5099E38544D9BF13054402EF10DD
:100C9000707675D9E30909FE85472320F900E5B789
:100CA000397106DE22DC26DA4AD84ED652D456D224
:100CB00032C66302051C638A051AB68AAE892A8485
:100CC000EF20001611E5B24781C77370043001A010
:100CD000EF20C0291C5C63920714B247638E070A99
:100CE0002808EF204004FD5413094402130A0401AC
:100CF000EF20002AEF10400CEF2040277C40639447
:100D00009700232204043C446394970023240404A2
:100D1000EF2000286C002808EF200003631305185B
:100D2000EF20C0241C5CADCFEF208026EF200024F4
:100D30003C44634FF00039A84A85EF10B06B19C1ED
:100D4000EF20800B3C44FD173CC43C446354F0004E
:100D50005C50FDF324C4EF20A023EF2020217C4031
:100D6000634FF00039A85285EF10D06819C1EF2009
:100D7000A0087C40FD177CC07C406354F0001C48F8
:100D8000FDF364C0EF20C020EF100028EF20001E0C
:100D90001C5CC1E7B247A9FFEF20801F014555A0A9
:100DA000EF20001F1C40DDC7B2454A85EF105046BA
:100DB000EF20C01B3C44634FF00039A84A85EF1078
:100DC000706319C1EF2040033C44FD173CC43C4410
:100DD0006354F0005C50FDF324C4EF20601BEF204F
:100DE000E0187C40634FF00039A85285EF10906006
:100DF00019C1EF2060007C40FD177CC07C4063542B
:100E0000F0001C48FDF364C0EF208018EF10C01FF5
:100E100031C9EF20A0151C5CB5DFCE852285444486
:100E2000EFF04FF7639C0A041C5C1840FD171CDCB4
:100E300001E7EF20601A48C01C48A1EFEF204015E1
:100E40000545F2506254D2544259B259225A925A2C
:100E500021618280EF2080114840EF10707EEF20EA
:100E6000201399B7EFF08FDA6DB73C41E38707E4C1
:100E70007370043001A07370043001A05C5044C44E
:100E8000D5DF13054402EF10F0564DD9EFF00FD81F
:100E900075B713050401EF10F0558547E310F5FA17
:100EA000F5B72285EFF0EFF0EF100016014551BFC6
:100EB0001DC9411122C44AC006C626C244412E891A
:100EC0002A84EF1030756383A40281464A868145E7
:100ED0002285F93385476300F502B24022449244EB
:100EE0000249410182807370043001A05C440545D1
:100EF00085075CC4DDB75C4485075CC4F9BF15CDCC
:100F0000ADC9011122CC26CA4AC84EC652C42A8491
:100F100006CE3289AE89EFF04FDB1C5C2A8A814411
:100F200085E35285EFF00FDAF240624426854249AC
:100F3000D244B249224A056182807370043001A014
:100F4000304001CE4C445C40B2954CC463E4F500A3
:100F50000C404CC44E85EF30E00E1C5C7D57FD17F5
:100F60001CDC7C40638CE7007C40854485077CC0AA
:100F70004DBF3C41D9D77370043001A01C4899E3A0
:100F8000854445B713050401EF10D04675D9E30930
:100F900009FE85472320F900E5B721C93C41A1CDD1
:100FA000A1CB011122CC26CA4AC852C42A8406CE3B
:100FB0004EC62E8AEFF06FD11C5C2A89814491CBFA
:100FC0008329C400D2852285EFF0CFDC8544232617
:100FD00034014A85EFF00FCFF24062442685424942
:100FE000D244B249224A056182807370043001A064
:100FF0007370043001A0EDDF7370043001A001E5CF
:101000007370043001A0411122C42A8406C6EF1077
:10101000F075005CEF10D077B24022852244410188
:10102000828001E57370043001A0411106C622C41C
:101030002A84EF10B0731C5C405C1D8CEF1050755F
:101040002285B24022444101828019C1085D82801C
:101050007370043001A01DCD979703009387078418
:10106000D843630CE502D847630CE504D84B63070B
:10107000E504D84F6302E504D853630DE502D85761
:101080006308E502D85B6303E502D85F630EE50001
:101090006F2030757370043001A001470E07BA97B6
:1010A00023A007006F20F0731D47CDBF1947FDB780
:1010B0001547EDB71147DDB70D47CDB70947F9BF64
:1010C0000547E9BF684582806CC5828003450505F8
:1010D000828009C5085D1335150082807370043065
:1010E00001A019C51C5D485D1D8D1335150082805A
:1010F0007370043001A0978703009387277A984381
:1011000005C3984705C7984B05C7984F05C798531F
:1011100005C7985705C7985B15C7985F15C38280A8
:1011200001470E07BA978CC3C8C382800547D5BF55
:101130000947C5BF0D47F5B71147E5B71547D5B7FF
:101140001D47C5B71947F1BF9787030093870775F8
:10115000D8436308E502D847630BE502D84B630A1E
:10116000E502D84F6309E502D8536308E502D85772
:101170006307E502D85B6308E502D85F6303A70253
:10118000828001470E07BA9723A007008280054797
:10119000D5BF0947C5BF0D47F5B71147E5B7154797
:1011A000D5B71D47C5B71947F1BF411122C426C2A3
:1011B0004AC02A8406C6AE843289EF10305B78407C
:1011C000FD576314F700232204043844FD576314C9
:1011D000F70023240404EF10B05B1C5C99E74A86F7
:1011E000A68513054402EF10B015EF1030583C44AB
:1011F000635BF0025C5085CB9304440209A83C4435
:10120000FD173CC43C446350F0025C5089CF2685F6
:10121000EF10501E6DD5EF10303E3C44FD173CC41E
:101220003C44E344F0FEFD573CC4EF107056EF1011
:10123000F0537C40635BF0021C4885CB93040401AF
:1012400009A87C40FD177CC07C406350F0021C481C
:1012500089CF2685EF10101A6DD5EF10F0397C403C
:10126000FD177CC07C40E344F0FEFD577CC0224467
:10127000B2409244024941016F10905197F701002A
:101280009387C739944317F701001307E7371843CB
:10129000C8C2636EE502411122C406C617F70100F9
:1012A000130787372A8408438C439105EFF04FA931
:1012B00097F70100938787339C436376F40097F791
:1012C000010023A58732B24022444101828017F7F2
:1012D00001001307273408438C4391056FF04FA694
:1012E00097F7010093878733984394437C43FD1716
:1012F0007CC3FC4299E37360043082801DC1797124
:101300004ECE56CA06D6BE8A22D426D24AD052CC57
:101310005AC85EC69147BA8963F8E7007370043013
:1013200001A07370043001A02A8BAE843289B68B81
:10133000428A6308082213050006EF2070382A84C9
:10134000630C05200A09232845034A869305500AA1
:101350005285EF20305D03C704001C587119230A21
:10136000E40203C704003E991379C9FF79C783C714
:101370001400A30AF40283C71400E1C383C7240046
:10138000230BF40283C72400CDCB83C73400A30B07
:10139000F40283C73400D5C383C74400230CF4028E
:1013A00083C74400D9CB83C75400A30CF40283C77E
:1013B0005400C1C783C76400230DF40283C76400CF
:1013C000ADCF83C77400A30DF40283C77400B5C703
:1013D00083C78400230EF40283C78400B9CF83C778
:1013E0009400A30EF40283C79400A1CB83C7A4008A
:1013F000230FF40283C7A400A9C383C7B400A30FBB
:10140000F40283C7B40095CB83C7C4002300F4045F
:1014100083C7C4009DC383C7D400A300F40483C75B
:10142000D40081CF83C7E4002301F40483C7E40020
:1014300089C783C7F400A301F404130A440052854A
:10144000A30104042326340323283405232A040497
:10145000EFF02F8D13058401EFF0AF8C9547B38724
:101460003741232C040400C81CCC40D023220404A0
:10147000232E04045E86DA854A85EFF0AF8508C026
:1014800063840A0023A08A007370043017F90100F6
:10149000130909178327090097F40100938404189E
:1014A00091C798409C407C4385077CC317F7010097
:1014B0001307C7151C43850797F6010023A8F614E8
:1014C0009C40CDCB8327090089EB9C40DC5763E629
:1014D000F90097F7010023A3871497F7010093877A
:1014E00027119C4317F701001307C71148541843ED
:1014F000850797F6010023ADF60E3CC46376A7007E
:1015000097F7010023A0A710D145EF50E06F97F7A0
:1015100001009387E7223E95D285EFF0EF80832785
:10152000090089C79C40FC436395070E8327090087
:10153000054499C79C40DC5763F43701EFE01FED89
:101540002285B250225492540259F249624AD24A38
:10155000424BB24B456182805285EF2090287D54EA
:10156000C5B713152600EF20B0152A8AE31505DC50
:101570007D54F9B797F7010023A2870A18438547DE
:10158000E31DF7F417F501001305851BEFE03FF8A5
:1015900017F501001305051CEFE07FF717F50100B3
:1015A0001305851CEFE0BFF617F501001305051DB7
:1015B000EFE0FFF517F501001305851DEFE03FF59E
:1015C00017FB0100130B0B1E5A85EFE05FF497FA2F
:1015D0000100938A6A1E5685EFE07FF317F501003C
:1015E0001305C51EEFE0BFF217F501001305451FF7
:1015F000EFE0FFF117F501001305C51FEFE03FF124
:1016000097F7010023AA670197F7010023A4570168
:10161000E9B5984094407C43FD177CC3FC42E397B6
:1016200007F07360043019B7411122C406C626C200
:101630004AC02A847370043097F40100938444FCF8
:101640009C40F9E311E497F70100938727FD80435D
:10165000130944004A85EFE0BFF11C5489C7130504
:101660008401EFE0FFF0CA8517F501001305451767
:10167000EFE09FEB97F70100938787F9984397F77F
:1016800001009387E7F69C43050797F6010023A125
:10169000E6F89840850797F6010023ABF6F401CBF6
:1016A00097F70100938787F79843784349EF9C4069
:1016B000B1C797F70100938767F69843630F8708D0
:1016C00073700430984039EB17F701001307C7F423
:1016D00014439442A5E27D5797F6010023A8E6F053
:1016E000984009CF9843784311CB984394437C4367
:1016F000FD177CC3FC4299E373600430B24022447E
:10170000924402494101828097F70100938707F1D3
:1017100098439C437C4385077CC32DB794439843EF
:10172000F8420507F8C217F701001307E7EE144364
:101730009442D5D2184358475847584397F601006A
:1017400023A6E6EA71BF984394437C43FD177CC30C
:10175000FC42B1FF7360043099BF97F70100938793
:10176000A7E89C4381C77370043001A02244B240B3
:101770009244024941016FE07FC941C517F701005A
:101780001307C7E914438147638BA606411106C6B8
:1017900022C426C27370043097F60100938646E691
:1017A0009C4291C710431C437C4285077CC29C42EB
:1017B000AA84404981C71C43FC43B9E797F701005D
:1017C000938787E59C43638A870497F70100938793
:1017D00067E49C436383870497F70100938787013D
:1017E0006308F40297F70100938787FF6300F40210
:1017F0008547B240224492443E85410182803E8525
:1018000082807370043001A0E13C4DBF9147D5B791
:101810009C5493B717008907E9BF8947D9BF7370F4
:10182000043097F701009387A7DD984309EF15C5AA
:101830009C43485581CB97F70100938727DE984357
:10184000784315E3828017F70100130727DD14435F
:101850001843F8420507F8C261FD17F701001307A6
:10186000E7DB0843F1B7984394437C43FD177CC3FF
:10187000FC42E9FB736004308280411122C42A8457
:1018800006C6EFE09FC411E497F70100938707D9DC
:1018900080434054EFE01FC3B240228522444101FF
:1018A0008280914763F5B7007370043001A0011185
:1018B00022CC06CE26CA4AC84EC652C42A847370A9
:1018C000043017F901001309A9D383270900CDEFCC
:1018D00071C43C486388F50817F70100130707D463
:1018E00063FCB7001443638B860C18434457B3B4AE
:1018F000950093C4140029A00443818C93B4140070
:1019000058546383E70A1C4C2CC863C607009547EC
:10191000B385B7400CCC93172700BA97584897F96E
:1019200001009389E9E18A07CE97631AF702130A47
:1019300044005285EFE0DFC397F70100938787CC1F
:1019400048549C4363F6A70097F7010023ACA7CA4D
:10195000D145EF50602BD2854E95EFE0FFBC99C08A
:10196000EFE0DFAA8327090081CB97F70100938777
:10197000E7CA9C43FC439DEBF2406244D244424997
:10198000B249224A0561828097F70100938707C90F
:1019900098439C437C4385077CC305FC97F7010073
:1019A0009387C7C7804335B74CD4B1BF6244F24078
:1019B000D2444249B249224A05611DB2814489B7E5
:1019C00025C1011126CA97F40100938424C59C40C7
:1019D00006CE22CC4AC84EC6638DA702737004306F
:1019E00017F901001309C9C18327090091C798405D
:1019F0009C407C4385077CC3584997F70100938737
:101A000067DF6302F7028327090081C79C40FC431C
:101A1000A5EBF2406244D2444249B249056182805A
:101A20007370043001A01C5517F70100130707DA83
:101A3000E38BE7FCE9FB930945002A844E85EFE040
:101A40003FB397F701009387E7BB48549C4363F685
:101A5000A70097F7010023A7A7BAD145EF50C01AF6
:101A600097F701009387C7CD3E95CE85EFE0DFABBA
:101A70009C405854DC57E368F7F8EFE03F9961B7B2
:101A80006244F240D2444249B249056191B815CD51
:101A9000011122CC26CA4EC62A8406CE4AC8EFE0DF
:101AA000DFA2584897F701009387C7D4AA898144D9
:101AB0006300F7024E85EFE0FFA0F2406244268506
:101AC0004249D244B249056182807370043001A05A
:101AD0001C5417F50100130565CFE38DA7FCF9FB36
:101AE00097F70100938747B09C43A9EB97F7010054
:101AF0009387C7B29C43445413094400DC574A857A
:101B0000B3B4F400EFE0DFA697F70100938787AF47
:101B100048549C4393C4140063F6A70097F7010050
:101B200023A2A7AED145EF50200E97F7010093876F
:101B300027C1CA853E95EFE03F9FADBF9305840165
:101B4000EFE09F9E85BF0111056506CE22CC26CA17
:101B50004AC84EC652C456C2EF208036630E051CDA
:101B6000AA8413050006EF20A0352A84630A051E07
:101B700005669305500A04D92685EF20A05A04581B
:101B80008567F117BE94B7474C45938797449309EF
:101B900044005CD84E85230C0402A30104042326D0
:101BA000040223280404232A0404EFE09F9713056A
:101BB0008401EFE01F979547232C0404F19800C897
:101BC0001CCC40D023220404232E04040146971584
:101BD00000009385E5B12685EFE0DF8F08C07370C4
:101BE000043017F901001309A9A18327090097F40C
:101BF00001009384A4A291C798409C407C43850730
:101C00007CC317F70100130767A01C43850797F6ED
:101C1000010023ADF69E9C40C9C38327090081EBD8
:101C20009C40DC5789E797F7010023A9879E97F727
:101C300001009387E79B9C4397F601009386869C5F
:101C400058549442850717F601002323F69A3CC4A2
:101C500063F6E60097F7010023A6E79A931727009B
:101C6000BA978A0717F50100130585AD3E95CE8515
:101C7000EFE09F8B8327090081C79C40FC43F1E77D
:101C80008327090091C39C40EF10F0498547630406
:101C9000F50E5DE17370043001A097F7010023AFEA
:101CA000879618438547E314F7F817F501001305E5
:101CB00025A9EFE0DF8517F501001305A5A9EFE0E1
:101CC0001F8517F50100130525AAEFE05F8417F5BE
:101CD00001001305A5AAEFE09F8317F50100130586
:101CE00025ABEFE0DF8297FA0100938AAAAB568515
:101CF000EFE0FF8117FA0100130A0AAC5285EFE00A
:101D00001F8117F50100130565ACEFE05F8017F543
:101D100001001305E5ACEFE08FFF17F50100130597
:101D200065ADEFE0CFFE97F7010023A7578F97F738
:101D3000010023A1478FE5BDF2406244D2444249ED
:101D4000B249224A924A05618280984094407C437D
:101D5000FD177CC3FC42E39507F2736004300DB7B6
:101D60006244F2404249B249224A924A2685D2440C
:101D700005616F20002773700430FD5717F70100CD
:101D80002326F786624497F7010023ABA786F2402B
:101D9000D2444249B249224A924A97F7010023A508
:101DA000078605616FE0EFCF7370043097F701008D
:101DB00023A807846FE02FDD17F701001307C78200
:101DC0001C4385071CC382807370043097F70100A1
:101DD00093870783984305E317F701001307C7822A
:101DE00008439C4381CB97F701009387278398434F
:101DF000784301EF828017F701001307278214430D
:101E00001843F8420507F8C2C1BF984394437C4386
:101E1000FD177CC3FC42F9FF7360043082804111DE
:101E200006C622C4EFE06FEA97E701009387C77DFB
:101E30008043EFE02FE9B2402285224441018280B5
:101E400097E701009387877C88438280797106D663
:101E500022D426D24AD04ECE52CC56CA5AC85EC6DA
:101E600097E70100938747789C43B1EF17E701009C
:101E7000130787791C43850797E6010023A6F678A8
:101E8000832A0700638F0A0697E701009387077686
:101E90009C43814463F1FA0897F901009389498AC8
:101EA00017EA0100130A8A7783270A008546D85764
:101EB00093172700BA978A07BE9983A7090063FF83
:101EC000F600854421A897E70100938727739C4378
:101ED0008144850717E701002322F77297E7010085
:101EE000938787719C4391C38544B25022542685C1
:101EF00002599254F249624AD24A424BB24B45616E
:101F0000828017E40100130424711C409C43DDC34C
:101F10007370043001A017E401001304E46F97F913
:101F200001009389E98117EA0100130A2A6F17EB70
:101F30000100130B2B6D1C409C43B5C31C40DC47B8
:101F400003A9C70083274900930B49005E8563EE10
:101F5000FA04EFE0EFE1832789021305890199C3B1
:101F6000EFE00FE18327C90203270B00DE851395FD
:101F700027003E950A054E956376F70017E70100A6
:101F80002322F768EFE04FDA83270A000327C9020C
:101F9000DC57E362F7FA1C4085449C43C5F3FD57C8
:101FA00017E701002324F76401B717E70100232F87
:101FB000F762DDBD17E701001307C7651C40184332
:101FC00097E6010023AAE66417E701002324F764DB
:101FD00097E70100938707629C43850717E7010095
:101FE000232AF7601C409C4399E7FD5717E701003F
:101FF000232EF75E51BD1C40DC47DC47DC4317E76E
:1020000001002325F75E49B597E701009387C75D77
:10201000984301E77370043001A0011106CE22CC71
:1020200026CA4AC84EC652C456C25AC0737004303B
:1020300097E401009384C45C984061EB98437D175A
:1020400097E6010023A2E65A9C43D9EB97E70100EB
:102050009387C75B9C43C9C797EA0100938A4A6E7E
:1020600017EA0100130A0A5A17E901001309095B6C
:10207000854919A83385EA00EFE00FCB83270900D3
:102080005854DC576379F70483A7CA08C1CF83A7E4
:102090008A09C04713058401EFE08FCD130B44007C
:1020A0005A85EFE0EFCC5C5483260A00DA8513955D
:1020B00027003E950A052A875695E3FDF6FA17E7AD
:1020C00001002321F754EFE02FC68327090058545D
:1020D000DC57E36BF7FA97E7010023AF37516DB791
:1020E00001449C4081CB97E70100938727539C4391
:1020F000FC4395E72285F2406244D2444249B2490A
:10210000224A924A024B0561828017E701001307B9
:10211000E75014431843F8420507F8C205B7EFF03B
:102120002F9CC9BF17E401001304444D1C4095C304
:102130001C40054999CF193B09C597E7010023AD1C
:10214000274B1C40FD1717E701002329F74A1C40C5
:10215000FDF397E701009387274A98438547E311EA
:10216000F7F8EFE0AFAA0544ADBF11CD81E573707C
:10217000043001A017E70100130707471C4399C764
:102180007370043001A07370043001A0411122C4A7
:1021900006C614431841850617E601002326D644D7
:1021A00097E601009386464694423304B70000C187
:1021B00063F7E602637FE40063FD860097E70100B2
:1021C0009387C74588431105EFE08FBA2285EFF06A
:1021D000EF8A1D3D01C9B240224441018280E36F74
:1021E000E4FCD9BF2244B24041016FE02FA211C9E3
:1021F00017E701001307473F1C4391C77370043072
:1022000001A06FE0AFA0411106C622C41843AA87FF
:10221000050797E6010023A9E63C97E601009386AF
:10222000E63F17E701001307273E184388423304AF
:10223000F7001105EFE0CFB32285EFF02F84E933EB
:1022400011E52244B24041016FE04F9CB24022446C
:1022500041018280411122C406C697E7010093879D
:10226000A7389C430144850717E70100232EF73662
:1022700097E70100938787399C4363E3F50C17EEDA
:102280000100130E6E5197E201009382A24A0144AD
:102290000147854F1303500A21A0311E6387C20DE9
:1022A00083278EFFBA85F5DB8327CEFFDC43232E01
:1022B000FEFE6382C71B03AFC700DC432A97814E33
:1022C000232EFEFE6385C70783A8C70093874803B4
:1022D000232017015CC383A788042326F7011CC7AA
:1022E00083A7C8021CCB83A70805232C07005CCB5F
:1022F00003A8080383470800639A6704C287850719
:1023000083C60700B3850741E38B66FE8981C2055A
:10231000C181231EB700850E1307070263001F0546
:102320008327CEFFDC43232EFEFEE39FC7F98327DE
:102330004E00232EFEFE49BF1A9419C22320060028
:10234000E1312285B2402244410182808145231E31
:10235000B700850E13070702E3141FFD76941317C9
:102360005400311EBA85E39DC2F397E701009387BD
:10237000A72A03AE070083270E00FDE397E70100BD
:102380009387472903AE070083270E00639807163B
:1023900017EE0100130ECE3A83270E0A639D071E27
:1023A00083274E0BD9DB83278E0B97EE0100938E8C
:1023B000EE44DC4317E701002320F7446381D73361
:1023C00083AFC700DC433307B500014397E6010044
:1023D00023A4F6420D4F89429308500A6386D7071B
:1023E000C8479307450308C35CC33C452326E70160
:1023F0001CC75C551CCB1C5599C3232657003C4970
:10240000232C07005CCB0328050383470800639552
:10241000172BC287850783C60700B3850741E38B67
:1024200016FF8981C205C181231EB700050313076A
:102430000702E383AFF083278E0BDC4397E60100AE
:1024400023ACF63AE39ED7F983270E0C97E60100FA
:1024500023A4F63A71B783274E00232EFEFEA1BDBA
:1024600083274E00130F8E00D4432322DE00638C9B
:10247000E625B307E500D84283A2C600814E232299
:10248000EE00894F1303500A6305EF068328C70047
:102490001387480323A01701D8C303A7880423A6E2
:1024A000F70198C703A7C80298CB03A7080523AC78
:1024B0000700D8CB03A80803034708006318671C6C
:1024C0004287050783460700B3050741E38B66FE95
:1024D0008981C205C181239EB700850E93870702BB
:1024E000638E121B83264E00D8422322EE00E31F88
:1024F000EFF80327CE002322EE0049BF83274E00CA
:10250000130F8E00DC432322FE006389E71B83A2A6
:10251000C700DC43AA95814E2322FE00894F130396
:10252000500A6305FF0683A8C7009387480323A0CA
:102530001501DCC183A7880423A6F5019CC583A7E8
:10254000C8029CC983A7080523AC0500DCC903A801
:1025500008038347080063976710C287850783C60F
:10256000070033870741E38B66FE098342074183F7
:10257000239EE500850E93850502638D120F832748
:102580004E00DC432322FE00E31FFFF88327CE002A
:102590002322FE0049BF83274E0A17EF0100130FC5
:1025A000AF24DC4317E70100232EF7226382E713F1
:1025B00083A2C700DC43AA95814E17E701002323BD
:1025C000F722914F1303500A6387E70783A8C700D8
:1025D0009387480323A01501DCC183A7880423A6A1
:1025E000F5019CC583A7C8029CC983A7080523AC35
:1025F0000500DCC903A80803834708006394670447
:10260000C287850783C6070033870741E38B66FED1
:10261000098342074183239EE500850E93850502C9
:10262000638A120383274E0ADC4317E70100232B3A
:10263000F71AE39DE7F98327CE0A17E70100232362
:10264000F71A69B70147239EE500850E93850502B9
:10265000E39A12FD83274E0B769493155400E38E74
:1026600007CC91B30147239EE500850E93850502B3
:10267000E39712F117EE0100130E8E0C83270E0A5A
:10268000769493155400E38D07D031B78145239E8E
:10269000B700850E93870702E39612E597E70100DE
:1026A000938747F703AE070076949315540083276A
:1026B0000E00E38F07CC99B58145BDB38327CE00CB
:1026C0002322FE00A9B58326CE002322DE0055B3C7
:1026D0008327CE0A17E701002326F710D1BD8327F1
:1026E0000E0C17E701002329F710D9B9797126D20A
:1026F0004AD04ECE52CC56CA5AC85EC606D622D44E
:1027000097E90100938949EE17E90100130949038C
:1027100017EA0100130ACAEE97EA0100938A0AF049
:1027200097EB0100938B8BEE97E40100938444EECA
:10273000054B21A883A709000324090A850717E789
:1027400001002323F7EAC93011E89C40E5F783270D
:102750000900E37CFBFEEFD07FCBC5BF7370043074
:1027600083270A00B9E38327C90AC0471305440039
:10277000EFD01FE083A70B00FD1717E70100232709
:10278000F7E89C40FD1717E701002323F7E88327AC
:102790000A0089C783A70A00FC4385E30858EF10A5
:1027A00050042285EF10F0034DB703A70A0083A75A
:1027B0000A007C4385077CC37DB703A70A0083A674
:1027C0000A007C43FD177CC3FC42E9FB73600430C4
:1027D000F1B797E70100938727E19C43DDE74111BB
:1027E00006C622C426C297E7010023A707E017E721
:1027F00001001307A7E21C43B7A6A5A59386565A66
:102800009C5B8C43639BD500D0436318B600944710
:102810006395C600DC476388D70008430C43938563
:102820004503EF20B00017E701001307A7DD1443AD
:1028300017E401001304C4F011A81C43A9CF1C43E2
:10284000FD1797E6010023AFF6DA144393972600AD
:10285000B6978A07A2979C43EDD3084393172500A8
:10286000AA978A073307F4005443A107A297C442EA
:1028700044C36385F402DC44B240224417E70100FC
:10288000232EF7D8924441018280854717E7010043
:102890002324F7D682807370043001A0C440D14550
:1028A000EF408036229544C1F9B701114AC806CEDF
:1028B00022CC26CA4EC62A897370043097E40100E0
:1028C000938404D49C4017E40100130424D5D9E771
:1028D0006314090003290400930949004E85EFD0D1
:1028E0003FC98327890289C713058901EFD05FC8D3
:1028F000CE8517E501001305E5EFEFD0FFC29C4040
:1029000081C71C40FC43ADE31C40638B27079C4000
:102910009DCF737004309C40C1EB97E70100938713
:10292000A7CF9843184325EBFD5717E70100232F46
:10293000F7CA9C4089CF1C40FC4391CB18401440FF
:102940007C43FD177CC3FC4299E373600430F24082
:102950006244D2444249B2490561828018401C4019
:102960007C4385077CC3ADB7184014407C43FD17FA
:102970007CC3FC42D1FB736004301C40E39927F90F
:102980009C40A1C397E70100938707C69C43ADCB4A
:102990007370043001A09C43DC47DC47DC4317E73D
:1029A00001002325F7C471B718401C407C438507FC
:1029B0007CC397E70100938727C6984318432DD718
:1029C000D9BF97E70100938767C417E70100130792
:1029D00027D79C430327470B631DF700F24062444F
:1029E00097E7010023AC07C2D2444249B2490561CE
:1029F00082806244F240D2444249B2490561D1BB6F
:102A00006244F240D2444249B24905616FD01FA0EE
:102A10003DC9411126C297E40100938424C04AC0F5
:102A20002E898C4006C622C4E105EFD07FB18840D4
:102A30001105EFD0FFB3FD57630AF90497E70100D2
:102A4000938787BC804398409C434A9440C3636CFF
:102A5000F40497E70100938727BC88438C409105D5
:102A6000EFD01FAE97E70100938747B89C4363768A
:102A7000F40097E7010023AB87B6B24022449244AA
:102A80000249410182807370043001A08C402244CD
:102A9000B2409244024917E501001305A5D59105FE
:102AA00041016FD07FA897E701009387A7B68843BD
:102AB00022448C40B24092440249910541016FD0BA
:102AC0003FA811C997E70100938707B29C4399E794
:102AD0007370043001A07370043001A0411126C24C
:102AE00097E40100938484B39840AE878C40B70686
:102AF0000080D58F06C622C41CCFE1053284EFD0FA
:102B0000BFA288401105EFD0BFA6FD57630EF400A9
:102B100097E70100938747AF8843B24092442295DC
:102B2000224441016FE08FF58C402244B240924430
:102B300017E50100130505CC910541016FD0DF9E1B
:102B400025CD411126C297E40100938424AD4AC0EB
:102B50002E898C4006C622C4E1053284EFD0DF9C6A
:102B600088401105EFD0DFA08547630AF40497E79A
:102B70000100938767A9804398409C434A9440C3CF
:102B8000636CF40497E70100938707A988438C409E
:102B90009105EFD0FF9A97E70100938727A59C4303
:102BA0006376F40097E7010023A287A4B240224491
:102BB00092440249410182807370043001A08C402C
:102BC0002244B2409244024917E50100130585C230
:102BD000910541016FD05F9597E70100938787A327
:102BE000884322448C40B2409244024991054101FD
:102BF0006FD01F95411106C622C426C25C45C0474E
:102C000035CC930484012685EFD09F9697E7010089
:102C10009387879D9C43B5E7930444002685EFD0B6
:102C20003F9597E701009387E79D58549C4363F6CF
:102C3000E70097E7010023A7E79C93172700BA97BF
:102C40008A0717E501001305A5AFA6853E95EFD0CD
:102C5000BF8D97E701009387679C9C4358540145BB
:102C6000DC5763F8E700854717E701002326F7984C
:102C70000545B24022449244410182807370043081
:102C800001A0A68517E50100130545B4EFD0DF8943
:102C9000C9B797E70100938727959C4381E7737035
:102CA000043001A0411106C622C426C2B707008025
:102CB0004045CD8F1CC12DC4EFD09F8B93044400A1
:102CC0002685EFD0FF8A97E701009387A793585492
:102CD0009C4363F6E70097E7010023A5E79293176B
:102CE0002700BA978A0717E50100130565A53E95E9
:102CF000A685EFD07F8397E70100938727929C43B7
:102D000058540145DC5763F8E700854717E7010091
:102D10002324F78E0545B24022449244410182802B
:102D20007370043001A011CD97E701009387878C61
:102D3000984397E701009387278D9C4318C15CC196
:102D400082807370043001A055C1D1CD411106C6F7
:102D500022C42A877370043097E801009388488A58
:102D600083A7080091CB97E701009387278B9443B3
:102D70009C43FC428507FCC217E301001303C38890
:102D80009C4103260300FD560144638FD70217EED2
:102D90000100130E2E8603250E000328070054435E
:102DA0006305A80005446371D6023308D640054484
:102DB000637CF80003250E00918F03260300B6976D
:102DC0009CC108C350C3014483A7080081CB97E787
:102DD00001009387A7849C43FC4381EF2285B24086
:102DE0002244410182807370043001A0737004306A
:102DF00001A0EFE0EFCEDDB7854717D70100232D07
:102E0000F77E828019C1684582800145828011C1A8
:102E10006CC5828097E70100938747808843828052
:102E200097D701009387C77D9C43054589CB97D7EA
:102E300001009387677B8843133515000605828060
:102E400031CD011126CA97D401009384247D9C4082
:102E500006CE22CC4AC84EC65855DC576379F702D5
:102E60001C4D63C707009C40D4579547958F1CCDD8
:102E700093172700BA97584917E901001309498C9D
:102E80008A07CA97630DF7009C40DC575CD5F24077
:102E90006244D2444249B2490561828082809309EA
:102EA00045002A844E85EFD0AFEC9C4017D7010037
:102EB000130747751843DC575CD46376F70017D7C0
:102EC00001002321F774139527003E9562440A05FB
:102ED000F240D244CE854A95B249424905616FD04D
:102EE000AFE419CD411106C622C426C297D701000E
:102EF0009387C77280436307A4007370043001A0F6
:102F0000014582807C4881E77370043001A05454ED
:102F10003848FD177CC86383E60099C70145B24075
:102F20002244924441018280930444002685EFD0DC
:102F30002FE4284897D701009387C76C984395479B
:102F4000898F48D41CCC6376A70097D7010023ABA8
:102F5000A76AD145EF30504B97D701009387477E42
:102F60003E95A685EFD04FDC054555BF7370043004
:102F700097D701009387C7689C4391CB97D70100EF
:102F80009387C76998439C437C4385077CC38280B1
:102F900097D701009387C7669C438DC397D70100DD
:102FA0009387C7679843784311CB984394437C43F6
:102FB000FD177CC3FC4299E373600430828097D78D
:102FC00001009387A7659043944398439547D4564F
:102FD000084E958F1CCF828097D701009387076496
:102FE000984309C79443F84A0507F8CA8843828082
:102FF00079714AD006D622D426D24ECE2A89737051
:10300000043097D401009384A45F9C4017D401003E
:103010001304C460BDE31C40BC4F89E71C40054756
:10302000F8CFD1E19C4081C71C40FC43F1EB7370A9
:1030300004309C408DEF1C40A84F11C56304090269
:103040001C4023AC07041C4023AE07049C4081C7EE
:103050001C40FC438DEBB250225492540259F24969
:103060004561828018403C4FFD173CCFE9BF1840B6
:103070001C407C4385077CC37DBF18401C407C43BB
:1030800085077CC349BF184014407C43FD177CC3AF
:10309000FC42F1F373600430B2502254925402594E
:1030A000F2494561828008402EC61105EFD04FCC11
:1030B000B245FD576380F50697D701009387C75443
:1030C00083A9070018409C43AE992322370163EC83
:1030D000F90497D701009387275488430C40910542
:1030E000EFD00FC697D70100938747509C4363F6F4
:1030F000F90097D7010023AB374FEFD02FB11DB7A1
:10310000184014407C43FD177CC3FC428DF3736070
:10311000043031BF0C4017D501001305A56D910592
:10312000EFD08FC0D9BF97D701009387A74E8843B0
:103130000C409105EFD0CFC0C9B779714AD04ECEBF
:1031400006D622D426D252CC2E89B289737004308E
:1031500097D401009384C44A9C4017D401001304FF
:10316000E44BF9EF18408947784F630CF7001C4097
:103170001345F5FFB84F798DA8CF1C400547F8CF10
:10318000ADE69C4081C71C40FC43F5E373700430FE
:103190009C40B1E7638609001C40BC4F23A0F900A6
:1031A000184085470145784F630BF7001C401349D1
:1031B000F9FF0545B84F3379E90023AC27051C40DA
:1031C00023AE07049C4081C71C40FC43C1E3B250BE
:1031D000225492540259F249624A45618280184051
:1031E0001C407C4385077CC375B7084036C6110573
:1031F000EFD00FB8B246FD576385F60897D70100A8
:103200009387874003AA070018409C43369A2322DD
:1032100047016363FA0897D701009387E73F884324
:103220000C409105EFD0CFB197D701009387073CB1
:103230009C436370FA0697D7010023A9473B91A8E6
:1032400018401C407C4385077CC329BF18401440AC
:103250007C43FD177CC3FC42BDFB73600430B2505D
:10326000225492540259F249624A456182801840C0
:1032700014407C43FD177CC3FC4289FB736004301F
:1032800031B70C4017D501001305C5569105EFD095
:10329000AFA9EFD0AF97F5B597D7010093878737E0
:1032A00088430C409105EFD0AFA9E5B751C141115A
:1032B00006C622C426C24AC07370043097D40100E7
:1032C000938404349C40B9EB99C23C4D9CC2B287B4
:1032D0008946704D74CD2E872A846386D70663FC99
:1032E000F6048D456387B70091456395B700630089
:1032F000D60C38CC8547630FF60405449C4081CB3F
:1033000097D70100938787319C43FC43A9E322852B
:10331000B2402244924402494101828097D7010081
:103320009387C72F98439C437C4385077CC369BF21
:103330007370043001A08546E39ED7FA3C4D33E715
:10334000B70038CD45BF3C4D85073CCD65B7EFD0C4
:103350003FF975BF130944004A85EFD06FA197D795
:1033600001009387272A48549C4363F6A70097D708
:10337000010023A9A728D145EF30100997D70100F4
:103380009387073C3E95CA85EFD00F9A1C5481C79E
:103390007370043001A097D70100938727289C43BE
:1033A0005854DC57E3FBE7F4EFD04F86B9B701443C
:1033B000B1B739CD011122CC26CA4AC84EC652C473
:1033C00056C206CEBA89368AB2842E892A84EFD0B4
:1033D000CF8FAA8A63050A003C4C2320FA00784C60
:1033E00089477CCC6389F40263F4970C8D4663872C
:1033F000D40091466396D400630AF70A232C24056F
:103400008547631EF7061C5499CB7370043001A0E6
:103410007370043001A03C4C85073CCCD5B797D7DE
:1034200001009387671C9C43ADEB93044400268501
:10343000EFD00F9497D701009387C71C48549C4343
:1034400063F6A70097D7010023AEA71AD145EF3046
:10345000A07B97D701009387A72EA6853E95EFD036
:10346000AF8C97D701009387671B9C435854DC5758
:1034700063F7E70063850900854723A0F900054449
:103480005685EFD02F842285F2406244D2444249CF
:10349000B249224A924A056182809305840117D578
:1034A00001001305A532EFD02F8865BF0144C9BFC5
:1034B0008547E397F4F43C4C33E92701232C24059A
:1034C00081B74DC1011122CC26CA2A844EC606CE30
:1034D0004AC8AE84EFC07FFF8947744C7CCC3C4C1B
:1034E0000547AA8985073CCC6395E6061C5481C72D
:1034F0007370043001A097D701009387E70E9C43B7
:10350000ADE7130944004A85EFD08F8697D70100B5
:103510009387470F48549C4363F6A70097D7010051
:1035200023A2A70ED145EF30206E97D701009387D5
:103530002721CA853E95EFC03FFF97D701009387AB
:10354000E70D9C435854DC5763F5E70099C0854765
:103550009CC06244F240D24442494E85B249056162
:103560006FC05FF67370043001A09305840117D516
:1035700001001305A525EFC03FFBC1B7AA8729C5E8
:103580007370043017D701001307870714439DE2B7
:10359000F04F894601456315D60023AE0704054563
:1035A0001C4381CB97D70100938747079843784303
:1035B00015E3828097D60100938646069042944296
:1035C0007442850674C2E9B797D70100938707054F
:1035D0009C437DB7984394437C43FD177CC3FC42D6
:1035E000E9FB7360043082805D71A6C2CAC052DC00
:1035F00056DA5AD85ED686C6A2C44EDE62D466D2E9
:103600006AD017D901001309690217DB0100130BF7
:103610002B0197D401009384E40097DA0100938A88
:10362000AA00054AA54B83270900984363010712A6
:10363000DC4783A90700EFE02FF8EFE0EFF88327DE
:103640000B002A8C6362F50A97D7010023AAA7FC16
:1036500001466370351B8840B3858941EFD0FFB4C4
:10366000EFE09F9A630105128840814601462C00D5
:10367000EFD00FE34DD9A247E3C807FEC24983A7A5
:10368000490189C713854900EFC09FEEEFE0CFF3F2
:1036900083270B002A8C636DF508A24717D701001A
:1036A000232087F9E3E2FBFCB317FA0013F70721A5
:1036B000631A071613F7770C6318071E93F70702B0
:1036C000C5D74E85EF00F01145B7DC47C04783AC46
:1036D0000700930944004E85EFC09FE95C502285A6
:1036E00082975C4C6384470B83270900984371FFE2
:1036F00003A70A0097D6010023A486F397D60100FA
:1037000023A4F6F297D7010023A2E7F2EFE0DF8FC0
:10371000A1BFDC47C04703AD0700930C440066859A
:10372000EFC01FE55C50228582975C4C6386470999
:1037300083270900984371FF03A70A0097D6010069
:1037400023A4F6EE97D7010023A2E7EEB9B7EFE086
:10375000AFE6EFE06FE783270B002A8CE366F5F80E
:1037600083A70A00884081499043B385894117D7D0
:103770000100232787EB13361600EFD01FA3EFE0DD
:10378000BF88E31305EEEFC07FC8F9BD1C4CCE85A2
:10379000E69763E9FC049C4089CF02CA66CC22CE3E
:1037A000EFF00FE88840814601464C08EFC03FFF2C
:1037B00005FD7370043001A01C4CE685EA97636C2C
:1037C000FD049C4089CF02CA6ACC22CEEFF04FE5BF
:1037D0008840814601464C08EFC07FFC31F9737088
:1037E000043001A0032509005CC000C8EFC05FD50C
:1037F000E5BDEFE07F8183270900DC47C047930CDC
:1038000044006685EFC0DFD65C4C638F47035C5095
:103810002285829791BD032509005CC000C8EFC0D6
:103820003FD239B7B24723ACF900A5CFE29723A224
:10383000F90023A8390193854900636FFC0403A5AF
:103840000A00EFC0FFCF0DB51C4C00C83387F9004C
:1038500058C0636DEC02330C3C416363FC029C4036
:1038600089CF02CA4ECC22CEEFF08FDB8840814652
:1038700001464C08EFC0BFF259F97370043001A043
:1038800003A50A00E685EFC0BFCB51B703250900A9
:10389000E685EFC0FFCAA5BF03250900EFC05FCAD8
:1038A000E1B37370043001A0B24783A6890123A855
:1038B00039013387D70023A2E9006364EC04B3071E
:1038C000FC4063EBD70483A749024E85829783A708
:1038D000C901E39B47D983A68901B2479840B697AF
:1038E00011CF02CA3ECC4ECEEFF08FD38840814636
:1038F00001464C08EFC0BFEAE31805D673700430E8
:1039000001A06374FC00E370F7FC032509009385B4
:103910004900EFC0FFC289BB03A50A009385490097
:10392000EFC01FC291B3411122C406C626C24AC0CD
:1039300017D40100130404CFEFF04FE31C4095CBE4
:10394000EFF00FE51C409DC38148014881470947BE
:1039500081461306004097D50100938525A61705DB
:1039600000001305A5C8EFD07F9939E973700430C2
:1039700001A017D90100130929E94A85EFC03FB911
:1039800097D40100938484E92685EFC05FB801468F
:10399000B145114597D7010023AA27C997D7010040
:1039A00023A497C8EFC09FD217D70100232CA7C626
:1039B00011CD97D501009385E59FEFD0CFF349B79F
:1039C000B240224492440249410182807370043023
:1039D00001A0A5C9797156CAAA8A1305C00222D4CA
:1039E00026D24AD04ECE52CC06D65AC85EC63A89A6
:1039F000B689328AAE84E9212A8405C9EFF00FD74F
:103A000097D70100938707C29C439DCFEFF04FD813
:103A1000130544002320540104CC232E4401232009
:103A2000340323222403EFC0DFAF2285B250225497
:103A300092540259F249624AD24A424BB24B456112
:103A400082807370043001A097DB0100938BCBDB85
:103A50005E85EFC0DFAB17DB0100130B2BDC5A8553
:103A6000EFC0FFAA0146B145114597D7010023AF2A
:103A700077BB97D7010023A967BBEFC03FC517D716
:103A800001002321A7BA01C997D50100938585922A
:103A9000EFD06FE6A5BF7370043001A039C50111E6
:103AA00022CC06CE26CA17D401001304A4B783285B
:103AB00004002A88014563850802BA842EC236872D
:103AC00032C442C6954663C5B602EFF06FB589476A
:103AD000630BF5020840814601464C00EFC03FCC25
:103AE000F2406244D244056182807370043001A0C8
:103AF0004C0081463A864685EFC0BFFFF2406244E3
:103B0000D244056182800840814626864C00EFC081
:103B10001FC9F9B719C1084182807370043001A030
:103B200001E57370043001A0411106C622C42A8445
:103B3000EFF0CFC348483334A000EFF06FC52285C3
:103B4000B24022444101828001E57370043001A03B
:103B5000411122C42A8406C6EFF04FC10050EFF095
:103B60002FC3B240228522444101828001E5737057
:103B7000043001A0411122C426C22E84AA8406C6A4
:103B8000EFF0CFBE80D02244B240924441016FF0AA
:103B90002FC04111714522C406C61D262A8411C5B5
:103BA000232005001105EFC09F962285B2402244D4
:103BB0004101828001CDB70700FFED8F81C773708F
:103BC000043001A099E57370043001A073700430D3
:103BD00001A0011122CC4AC84EC652C456C206CE1C
:103BE00026CABA893689B28A2E842A8AEFF04FA370
:103BF00011E5638509007370043001A0EFE0CF9BED
:103C000083240A00B37794006316090295C763877B
:103C10000A009347F4FFE58F2320FA00EFE0CFBEC0
:103C2000F240624426854249D244B249224A924A2D
:103C300005618280E30DF4FCE38209FEB335500197
:103C4000E20563050900B7070004DD8D4E86C18DCE
:103C500013054A00EFE0FFE6EFE00FBB19E1EFC00C
:103C6000EFFAEFF0CFB593176500AA8963D8070084
:103C7000B7040001FD14B3F499005DB7EFF00FAF86
:103C800083290A00B3773401631E090089CB638856
:103C90000A009347F4FFB3F737012320FA00EFF04F
:103CA0002FAFF9B7E31DF4FEDDB701C9B70700FF79
:103CB000ED8F99C77370043001A07370043001A0B8
:103CC000411122C42A8406C626C24AC02E89EFF0BA
:103CD000EFA904409345F9FFB3F795001CC0EFF03E
:103CE0002FABB24022442685024992444101828092
:103CF000411122C42A8406C6EFC02FFD0040EFC048
:103D00006FFCB240228522444101828009C93707F5
:103D100000FFB3F7E50099C77370043001A073701A
:103D2000043001A06F20D07BB70700FFF18F81C75F
:103D30007370043001A001E67370043001A001111A
:103D400022CC4AC84EC652C406CE26CA3689AE898F
:103D50002A8A3284EFF0CF8C21E163050900737069
:103D6000043001A0EFE04F8583240A00CE85528500
:103D7000B3E49900613FB37794006307F4068324AA
:103D80000A00EFE06FA8F240624426854249D2441F
:103D9000B249224A05618280EFE00F8283240A0043
:103DA000CE855285B3E434019537B3F78400638D33
:103DB0008702E30609FCB70500054A86C18D130595
:103DC0004A00EFE01FD0EFE02FA419E1EFC00FE4AD
:103DD000EFF0EF9E93176500AA8463DF0700B70733
:103DE0000001FD17FD8C45B783270A001344F4FF3B
:103DF000E18F2320FA0071B7EFF04F9783240A0078
:103E0000B3779400639787009347F4FFE58F2320EF
:103E1000FA00EFF0EF97E1B7411122C406C62A84F9
:103E200026C2EFD07FF95C4085C308489304C400E4
:103E30006316950015A0084863009502B7050002B7
:103E4000EFE03FE55C40E5FB2285612A2244B24079
:103E5000924441016FE04F9B7370043001A009C987
:103E6000370700FFB3F7E50099C77370043001A06E
:103E70007370043001A06F20B06601C9B70700FF5E
:103E8000ED8F99C77370043001A07370043001A0E6
:103E9000411122C426C206C62A84AE84EFF00F8DDB
:103EA000184093C7F4FFF98F1CC02244B2409244DB
:103EB00041016FF0EF8D19C1084D8280014582806C
:103EC000411122C406C62A84EFD01FEF97C7010014
:103ED000938707769C43A1EBE56717D7010013078B
:103EE0006795F11797C6010023AAE67417C701006A
:103EF0002324F77417D701002320F79497C70100F4
:103F00009387477317D701002326F792854717C772
:103F100001002327077217C70100232D077017C759
:103F200001002327F77019E8EFE00F8EEF10800FE4
:103F300001442285B240224441018280130584005D
:103F400093773500C1EFE5671307F5FFE917E3ED58
:103F5000E7FC97C601009386666E9C4229A09843B1
:103F600011C7BE86BA87D843E36BA7FE17C7010007
:103F70001307476CE38AE7FA9843414613848700A6
:103F800098C2D843B306A7406378D6023388A70007
:103F90002322D800C8C38325480097C60100938612
:103FA000E66911A0BA8698425043E36DB6FE23201D
:103FB000E80023A00601D84397C701009387076F45
:103FC0009C43998F17C701002322F76EEFE0CF8340
:103FD00031DC2285B2402244410182807199110571
:103FE0009DB729C9411122C406C62A84EFD0DFDC5F
:103FF000930584FF0326C4FF17C701001307076456
:1040000011A03E871C43D443E3EDC6FE232CF4FEEF
:104010000CC397C701009387676998438327C4FF40
:104020002244B240BA9717C701002321F768410123
:104030006FD09FFD828097C70100938727678843D1
:10404000828082803367B5000D8BAA871DE79308B5
:10405000D6FFAA982A87AE866371150303A80600C7
:1040600011079106232E07FFE36A17FF9347F5FF19
:10407000C697F19B9107BE95AA972A9663F3C70A44
:104080009386450013884700B3B6D70033B80501BF
:1040900033E7F50093C61600134818000D8BB3E6FE
:1040A000060113371700758F330EF64093861700FD
:1040B00029CF1337AE0031EB13532E002E88BE8666
:1040C0000147832808000507110823A0160191065F
:1040D000E36967FE1377CEFFBA95BA976302EE04E1
:1040E00083C60500138717002380D700637AC702B1
:1040F00083C6150013872700A380D7006372C70209
:1041000003C725002381E7008280B307F640AE97FE
:10411000850503C7F5FF8506238FE6FEE39AF5FEC6
:1041200082808280B367C5008D8BB308C500E9C368
:104130006371150FB307A0408D8B13873700954629
:1041400093F5F50F130815003383A8407D166373AC
:10415000D70015476363E60CD5CF2300B5000547AC
:10416000638DE700A300B5000D4713082500639693
:10417000E700130835002301B500139685004D8E26
:1041800013970501518F3303F34093968501D98E20
:1041900013562300AA97014794C305079107E36DBF
:1041A000C7FE1377C3FFB307E8006307E306238066
:1041B000B70013871700637C1703A380B70013872A
:1041C0002700637617032381B700138737006370D6
:1041D0001703A381B70013874700637A170123826F
:1041E000B7001387570063741701A382B70082805A
:1041F00093F5F50F13978500D98D139705014D8F12
:10420000E37715FFAA87910723AEE7FEE3ED17FFDB
:10421000828082802A8895B78280AA8749BF834797
:1042200005002A8799C7050583470500EDFF198D0D
:1042300082800145828005058347F5FF850503C718
:10424000F5FF91C7E389E7FE3385E7408280814728
:10425000E5BFAA87850503C7F5FF8507A38FE7FE9E
:1042600075FB828083460500930700026397F60082
:10427000050583460500E38DF6FE938756FD93F70B
:10428000D70F85C7AA87814585CE01458507138647
:1042900006FD1317250083C607003A9506053295DB
:1042A000F5F699C13305A0408280938536FD83469B
:1042B000150093B5150093071500E1FA0145D5B730
:1042C000014582809C412380A7009C4185079CC1B9
:1042D000828097C601009386E6369C4217570300FA
:1042E0001307475613861700BA972380A70097C570
:1042F000010023A9C534A9476308F500930700040A
:104300006305F6000145828075DE370610F005076B
:104310008347F7FF2320F6F09C42FD1797C5010065
:1043200023A2F532EDF7014582804D7123229114CD
:1043300023202115232A511323248113232611140A
:1043400023248114232E3113232C4113232861139A
:1043500023267113232291132320A113232EB1119D
:10436000AA842E8932C6130C5002A54A834709003D
:1043700063808703B9CB804011A0A1CB2300F40058
:1043800080400509050480C083470900E39787FF43
:104390000346190093081900C686130D0002FD5943
:1043A0007D5A0148130550059307D6FD93F7F70F83
:1043B000138916006363F52A17C70100130787C422
:1043C0008A07BA979C43BA9782878320C114032433
:1043D000811483244114032901148329C113032A5E
:1043E0008113832A4113032B0113832BC112032C46
:1043F0008112832C4112032D0112832DC111716191
:104400008280A14C02C4854763D50715B24780401E
:10441000938B770093F68BFF03AB060083A94600CE
:10442000938786003EC6668681465A85CE85EF20F4
:10443000A02D2AC8814763853723930D4101854B01
:10444000668681465A85CE85EF10504E8146668637
:104450002A8BAE89EF20402BA24723A0AD00938684
:104460001B00910D63843701B68BD9BFE37E9BFFA0
:1044700063DD4601A2872380A70180407D1A930750
:1044800014009CC03E84E3C846FF93962B001C0892
:10449000BE9631A8938777052300F4008040FD1B6A
:1044A00093871B00050480C0F116E351F0EC9C4299
:1044B000E3E2FAFE93870703C5B79C409306000327
:1044C00032472380D7009C4093064700C14C138697
:1044D000170090C013068007A380C700804002C465
:1044E000BA87050480C003AB0700814936C625BFE3
:1044F000B24783AC0700938B470063840C1C635F57
:1045000040199307D0026319FD1683C70C0085C3B9
:1045100063DC09189440850C7D1A2380F6008040E6
:10452000050480C083C70C00E5F7635D400180404F
:10453000930700022300F40080407D1A050480C028
:10454000E31A0AFE5EC61DB502C48547A94CE3CF37
:1045500007EBB24780409386470071B703C6160049
:10456000CA8699B59C40930650022380D7008040AC
:10457000050480C0E5BBC14C02C471B5B24703C697
:104580001600CA8683A9070091073EC6E35E0AE0CB
:104590004E8AFD5911BD03C61600130DD002CA86FE
:1045A00021B59347FAFFFD8703C61600337AFA0058
:1045B000CA86DDBB03C61600130D0003CA86EDB321
:1045C00083C51600930906FDCA86938705FD2E86CE
:1045D000E3EEFAFA93972900BE9985068609AE990B
:1045E00083C50600938909FD938705FD2E86E3F3B5
:1045F000FAFE69BF32479C40144311073AC6238034
:10460000D7008040050480C095B3854763D3070B6E
:10461000B24793867700E19A938786003EC683A9C6
:1046200046009C4263DC090A94401306D002B3079B
:10463000F0402380C6008040B336F000B30930411B
:10464000050480C03E8BB389D940A94C02C4E1BBAC
:1046500003C616000508CA8681BB9C40468921B75F
:10466000E37D9BDD8547814B8546E3C547E131BD51
:1046700097CC0100938C0CD5CE856685EF10405306
:10468000330AAA40635C400180402300A4018040BB
:104690007D1A050480C0E31A0AFE014A83C70C0094
:1046A000E38207EAE3C809E6FD197D57E394E9E6EA
:1046B000ADBDB247938647009C4336C693D9F741B8
:1046C00095B7635640019307D002E313FDFA97CCE8
:1046D0000100938C2CCF930780021DBD3E8BA94C0B
:1046E00002C4804089B34D71232E3113B7090040B5
:1046F0009387F9FF2324811423229114232C41133F
:10470000232A511323261114232021152328611352
:104710002326711323248113232291132320A11311
:10472000232EB1112A8A2EC417C40100130484F168
:10473000975A0300938A0A1197C40100938404A234
:104740003EC693055002294513080004B70610F031
:1047500083470A006386B704C1C71840050A1306D9
:104760001700569797C8010023AEC8EC2300F70046
:104770006382A706E31E06FD175703001307870C85
:1047800005078347F7FF23A0F6F01C40FD1717C667
:1047900001002329F6EAEDF783470A00E39EB7FA02
:1047A00083461A0013051A002A87930B00027D5BCB
:1047B0007D5C014893055005A5489387D6FD93F786
:1047C000F70F130A170063E7F5348A07A6979C438F
:1047D000A6978287175703001307C70655F28DBFA8
:1047E0008320C11403248114832441140329011458
:1047F0008329C113032A8113832A4113032B011335
:10480000832BC112032C8112832C4112032D011220
:10481000832DC11171618280A14C014D854763DBFD
:104820000719A2479D07E19B83AD070003AB470033
:10483000138787003AC4668681466E85DA85EF1055
:10484000B06C2AC863066D35130941018549668637
:1048500081466E85DA85EF10700D66868146AA8DD9
:104860002E8BEF10706A2320A90085091109E3102F
:104870006DFFE3FE9DFD13060004B70610F063D143
:1048800089031C4013871700D69797C5010023ABF7
:10489000E5DA23807701630CC7047D1CE3C389FF3D
:1048A000B2476800A548B386F9008A061C08BE9680
:1048B000294813030004370610F0E384A6E89C425D
:1048C0009305000363F4F800930570051840AE9754
:1048D00093051700569717CE01002325BED6230057
:1048E000F7006380072B638C6526F116F9B717571D
:1048F0000300130727F505078347F7FF23A0F6F00A
:104900001C40FD1797C5010023AEF5D2EDF77D1CC5
:1049100071B71C40130600041387170097C50100E8
:1049200023A2E5D2B386FA00930500032380B600E4
:104930006300C73E890797C6010023A5F6D05697A6
:10494000930680072300D70017570300130787EF4C
:10495000B70610F0639EC70005078347F7FF23A043
:10496000F6F01C40FD1717C60100232DF6CCEDF71D
:10497000A247C14C014D91072247014B832D0700EF
:104980003EC455BDA24783AC070013894700638F1F
:104990000C3A635480219307D002639EFB2E03C719
:1049A0000C00BA856310072025AC8547A94C014D42
:1049B000E3C907E7A2479107C1B7A247834617009B
:1049C000528703AB070091073EC4E3580CDE5A8CB4
:1049D0007D5BE5B383461700930BD0025287F1BB92
:1049E0009347FCFFFD8783461700337CFC0052870A
:1049F000E9B383461700930B000352877DBB034640
:104A00001700138B06FD5287930706FDB286E3EE6F
:104A1000F8FA93172B00DA9705078607B297034633
:104A20000700138B07FD930706FDB286E3F3F8FE3C
:104A300069BFA2451C402946984193861700D69726
:104A400017C501002320D5C02380E7001389450046
:104A50006301C72A930700046387F6204AC4D5B1CF
:104A6000854763DF0729A24713877700619B930778
:104A700087003EC4032B47001C43635B0B30184088
:104A8000130600049306170097C5010023ACD5BA9E
:104A900056979305D0022300B7006388C62CB3074E
:104AA000F0403337F000330B6041BE8D330BEB40E9
:104AB000A94C014D49B38346170005085287F5B943
:104AC000834617005287D5B91C409306000413870C
:104AD000170017C601002327E6B6D6971306500223
:104AE0002380C700E31FD7C417570300130787D5D8
:104AF000B70610F005078347F7FF23A0F6F01C4028
:104B0000FD1717C60100232FF6B2EDF71DB9C14CF2
:104B1000014D29B31C40930600042A8A138717000D
:104B200017C601002320E6B2D69713065002238051
:104B3000C700E318D7C0175703001307A7D0B7065D
:104B400010F005078347F7FF23A0F6F01C40FD1780
:104B500017C601002328F6AEEDF72A8ADDB61757EF
:104B60000300130727CE05078347F7FF2320F6F03E
:104B70001C40FD1797C5010023A6F5ACEDF7F11613
:104B80002DBB175703001307E7CBF1FDF11635B323
:104B9000E3FC9DCB8549C5B1014C03C70C00BA8528
:104BA000E30E07EAFD58294513080004B70610F084
:104BB00063570B0A1C4013861700D69717C30100D2
:104BC0002322C3A82380E7006384A50663040609A3
:104BD000850C03C70C007D1CBA8579FBE35080E986
:104BE0001C409305000213060004B70610F021A034
:104BF0007D1CE3050CE613871700D6972380B700CA
:104C000017C501002320E5A4BA87E313C7FE175791
:104C10000300130727C305078347F7FF23A0F6F018
:104C20001C40FD1717C50100232EF5A0EDF7C9B7ED
:104C300017570300130707C141DE05078347F7FF36
:104C400023A0F6F01C40FD1717C60100232CF69E8A
:104C5000EDF7BDBF175703001307C7BEF9BF7D1B94
:104C6000E31A1BF5A5BF175703001307A7BDB70627
:104C700010F005078347F7FF23A0F6F01C40FD174F
:104C800017C601002320F69CEDF74AC45DBC97BC13
:104C90000100938C2C73DA856685EF007071330CFC
:104CA000AC40E35C80EF1C4013060004B70610F034
:104CB00021A07D1CE3020CEE13871700D6972380FA
:104CC000770197C5010023AFE596BA87E313C7FEC6
:104CD00017570300130707B705078347F7FF23A0FC
:104CE000F6F01C40FD1797C5010023ADF594EDF7D4
:104CF000C9B7175703001307E7B4B5FA4AC491B40C
:104D0000A247138747009C433AC413DBF741B5B36E
:104D100017570300130707B3B70610F005078347BB
:104D2000F7FF23A0F6F01C40FD1717C60100232B48
:104D3000F690EDF7854717C701002325F7909307F5
:104D4000800717570300230FF7AE1DB1635680018C
:104D50009307D002E39DFBF297BC0100938C8C6615
:104D6000130780029305800235BD97560300938692
:104D700066AD370610F0850603C7F6FF2320E6F080
:104D800018407D1797C5010023AEE58A6DF701BB7A
:104D9000BE8DA94C014D45B4B70710F023A0A7F272
:104DA00001A03971130341022ED29A8506CE32D466
:104DB00036D63AD83EDA42DC46DE1AC62D32F2400A
:104DC0000145216182805D711303810322D42AC6CB
:104DD00032DC2A841A86680006D6BEC236DEBAC025
:104DE000C2C4C6C61ACEEFF04FD4B2472380070024
:104DF0003245B250018D225461618280B70710F0B4
:104E000083A647F403A607F403A747F4E31AD7FEE3
:104E1000856693868638B29633B6C600B305E6003B
:104E200023A4D7F423A6B7F48280B70710F003A712
:104E300047F403A607F483A647F4E31AD7FE856672
:104E400093868638B29633B6C60023A4D7F4B3054A
:104E5000E60023A6B7F49307000873A047308280CA
:104E6000797122D406D626D24AD04ECE52CC56CA1A
:104E70005AC85EC697B701009387477D17B40100F3
:104E80001304847C98431C40930647069387470687
:104E900017B60100232AF67A856717B60100232783
:104EA000D67A938777BB63CDD700B2502254925401
:104EB0000259F249624AD24A424BB24B4561828062
:104EC000FD779387C74A3E9797B7010023A0E778FD
:104ED0007D238547631DF504EF00D0078549114BFD
:104EE000814BA144314A814A2A896303350717B5AA
:104EF00001001305E54FEFF0DFEAEF00F03DD2844B
:104F00006306350717B5010013050551EFF07FE97A
:104F10002685EFF07FE82254B25092540259F249AC
:104F2000624AD24A424BB24B45616FC0FFE717B5A8
:104F300001001305A549EFF0DFE6EF00B001854958
:104F4000194B894BA944394A894A2A89E31135FB0F
:104F5000EF009038E31825FB639C0A00184089672E
:104F6000938777328144E3C5E7FA81B7DA844DB796
:104F7000DE8479BF17B501001305454C6FF07FE261
:104F800017B501001305054C6FF0BFE1411122C4B4
:104F900026C206C6856417B401001304244B938708
:104FA00084380100FD17F5FF2285EFF09FDFC5BFB4
:104FB000411106C6A929D125B24041016F007027D1
:104FC000411106C622C426C25D2985476313F50434
:104FD00091440144EF00007885476309F50017B557
:104FE00001001305E540EFF0DFDB2684EF00D02E53
:104FF0008547630AF50017B501001305E541EFF099
:105000005FDA136484002285B24022449244410155
:10501000828017B501001305653BEFF09FD89944D6
:1050200009444DBF7370043001A082807370043056
:1050300001A0797126D24AD04ECE52CC56CA5AC857
:1050400006D622D417BA0100130A4A6217BB010020
:10505000130B0B619304500505499309E00A930A69
:10506000E00B0145EFD07F84EFC01FD62A840325D3
:105070000A0081461306F00A6C0002C697B70100C9
:1050800023AC975CEFB0AFF109C597B7010023A738
:10509000275DEFC07FD3018D63F4A90063F6AA00FA
:1050A00097B7010023AC275B014597B7010023A503
:1050B000975AEFD08FFFEFC03FD12A8403250A0013
:1050C00081461306F00A6C0097B7010023A6975893
:1050D000EFB01FBD09C597B7010023A12759EFC045
:1050E000BFCE018D63F4A90063F6AA0097B7010053
:1050F00023A6275797B7010023A0975683270B00B5
:10510000850717B70100232DF754A1BF397126DA9F
:105110004AD84ED652D456D25AD05ECE62CC66CA47
:1051200006DE22DC6AC817BA0100130A2A5417B92E
:1051300001001309695297BB0100938BEB5297BC96
:105140000100938C2C52294C054B914A85499304BC
:10515000500502C401463314CC00EFC0FFC62A8DAF
:1051600003250A00814622866C00EFB07FB309C593
:1051700097B7010023A4374FEFC01FC53305A541E2
:105180009307F4006376850017B701002328374D95
:1051900063FDA724224697B7010023A1374D0506DA
:1051A00032C4E3DACAFA02C403250A008146014682
:1051B0002C00EFB0CFDE6306652597B7010023AF63
:1051C0003749A24785073EC4E3D0FAFE02C4014630
:1051D0003314CC00EFC05FBF2A8D03250A0081463F
:1051E00022862C00EFB0AFDB09C597B7010023A7DB
:1051F0003747EFC07FBD3305A5419307F4006376C1
:10520000850017B70100232B374563FAA71C2246F8
:1052100097B7010023A43745050632C4E3DACAFA7A
:1052200003A50B0097B7010023A80742EFC04FF971
:1052300083270900638997005145EFC05FFB8327EF
:105240000900E39B97FE5145EFC07FFA97B7010035
:1052500023A4074002C403250A00814601466C00CE
:10526000EFB01FA4814601462C006306650197B785
:10527000010023A5373F03250A00EFB04FD2914527
:105280006306650197B7010023AA373D832709000C
:1052900003A50B006396970097B7010023A0373D45
:1052A000EFC02FE083270900854503A50B00639617
:1052B000970097B7010023A3373BEFC08FDEA247CB
:1052C00085073EC4E3D9FAF883270900514563896D
:1052D0009700EFC0DFF1832709005145E39B97FE5C
:1052E000EFC0FFF097B7010023A8073602C40325DB
:1052F0000A00814601466C00EFB09F9A630D650F6E
:1053000097B7010023AC3735A24785073EC4E3D0E9
:10531000FAFE03A50B00EFC0AFEA832709006389FB
:1053200097005145EFC0BFEC83270900E39B97FE30
:105330005145EFC0DFEB97B7010023AF073002C440
:1053400003250A00814601462C00EFB04FC5814677
:1053500001466C006306650197B7010023A0373151
:1053600003250A00EFB0DF9391456306650197B707
:10537000010023A5372F8327090003A50B0063969F
:10538000970097B7010023AB372DEFC08FD183274C
:105390000900854503A50B006396970097B70100A8
:1053A00023AE372BEFC0EFCFA24785073EC4E3D92A
:1053B000FAF883270900514563899700EFC03FE35E
:1053C000832709005145E39B97FEEFC05FE283A767
:1053D0000C00850717B701002326F7289DBB22463E
:1053E000050632C4E3D6CADE25BD2246050632C410
:1053F000E3D3CAD64DBBA24785073EC4E3D9FAEE34
:1054000009BFA24785073EC4E3D0FADAC1B3411110
:1054100001469145154506C6EFB04FAB97B5010063
:105420009385050497B7010023A2A724EFB0BFCC52
:10543000814801488147094781461306004097B5D6
:1054400001009385250317050000130565CCEFB017
:10545000FFEAB2408148014897B701009387C7200F
:10546000054781461306004097B501009385050165
:1054700017050000130525BC41016FB03FE817B7C1
:1054800001001307271E97B601009386661D17B605
:1054900001001306E61B1C4310428C4217B50100A5
:1054A0001305451B0328050001456386C500B38726
:1054B00007413335F00097B701009387271A9C43C3
:1054C00094421843FD17B337F000B307F04017B606
:1054D0000100232FD6167D8D97B6010023ACE6166A
:1054E0008280011122CC06CE26CA4AC84EC652C4BA
:1054F00058419307A00A2A8404416309F7108146A2
:10550000014681452685EFB0AFF985476316F50062
:1055100097B7010023A2A71605498549032A04006D
:105520008146014681455285EFB08FF76304250B14
:105530009304800C8146014681455285EFB02FA629
:105540001C446300250D850717B701002326371378
:10555000FD141CC4E5F08146014681455285EFB03B
:105560000FA46316250197B7010023A72711032A6B
:1055700004008146014681455285EFB04FA2630089
:1055800025079304800C8146014681455285EFB082
:105590002FF11C44630A2505850717B70100232D49
:1055A000370DFD141CC4E5F0814601468145528546
:1055B000EFB00FEFE31425F7032A040081460146FC
:1055C0008145528597B7010023A8270BEFB04FED17
:1055D000E31025F797B7010023A0270B91BF97B7DA
:1055E000010023AB270971BF8507FD141CC4C1FC52
:1055F0008146014681455285EFB08FEAE31025F3DD
:1056000065BF8507FD141CC495F4B1B781460146FA
:1056100081452685EFB0AF9885476316F50097B7AB
:10562000010023ABA7041309800C8549814601467C
:1056300081452685EFB0CFE61C44630A3503850714
:1056400017B70100232A37037D191CC4E31009FE94
:105650002685814601468145EFB08FE485470440A9
:10566000E31FF5E897B7010023A8A70049BD850708
:105670007D191CC4E31C09FAE1BF41119305800C9C
:105680001305800C06C622C4EFB04F8E9747030067
:1056900023AAA71E9307A00A174703002326F71E75
:1056A00081451305800C9747030023A1071EEFB027
:1056B000EF8B9747030023ADA71C9747030023AB4D
:1056C000071C174403001304E41B9747030023A59A
:1056D000071C084097B501009385C5DAEFB0BFA15C
:1056E000484497B501009385E5DAEFB0DFA01C4090
:1056F000A1CF81480148814701479746030093861F
:1057000066181306004097B501009385A5D91705C3
:105710000000130545DDEFB07FBE2244B240814852
:105720000148814701479746030093866616130692
:10573000004097B50100938565D717050000130554
:1057400085DA41016FB09FBB5C44C5F7B24022448B
:105750004101828017B70100130707F210439747F2
:1057600003009387271217B701001307A7F0184308
:10577000944701456389E60098471335160097B6AC
:10578000010023A9E6EE17B70100130767EED44B1B
:1057900018436388E600DC4B17B70100232AF7ECB7
:1057A000828001458280797122D426D24AD04ECEA1
:1057B00052CC56CA5AC85EC662C406D697B4010017
:1057C000938484EE97B90100938949EC17BA0100DC
:1057D000130A8AEB97BA0100938A4AEC97BB01003F
:1057E000938B0BEC17BC0100130C8CEA05440D499C
:1057F000094B88408145EFB0AFEBE31C85FE03A564
:105800000900EFB09FF7631C250B03250A00EFB0DA
:10581000DFF66313250B83A70A006387870097B71A
:10582000010023A187E8F1B783A70B00E39987FE66
:1058300083270C0003250A00850717B701002329D9
:10584000F7E4EFC0EF9703A50900EFC06F9783A7B8
:105850000A006387870483A70B00638387040145DD
:10586000EFB0FFFB6317650503A50900EFB0FFF07C
:10587000631D650503250A00EFB03FF0631465055D
:105880008840EFB0AFA26306850097B7010023AB55
:1058900087E00145EFB0BFF829DD7370043001A047
:1058A000014597B7010023AF87DEEFB05FF7E30D47
:1058B00065FB7370043001A07370043001A0737035
:1058C000043001A07370043001A07370043001A093
:1058D000011122CC26CA4AC84EC652C406CE17B9F8
:1058E0000100130969DC17BA0100130A6ADB97B4D7
:1058F0000100938424DA97B901009389E9D905441A
:105900002DA097B7010023AF87D89C4003A70900BB
:1059100085076386E70097B7010023A587D89C40D9
:10592000850717B701002327F7D603250900F95586
:10593000EFB00FD8E31785FC83270A00E39387FCB9
:1059400003250900EFB08F966306850097B7010025
:1059500023AA87D4014597B7010023A187D4EFC0BC
:10596000DFF497B7010023AB07D245B701114AC84E
:1059700017B90100130949D30325090022CC4EC6EB
:1059800006CE26CA054497B901009389E9D0EFB045
:10599000EF9163058508A94403250900A145EFB0EF
:1059A0002FD163028508FD14514597B7010023AB41
:1059B00087CEEFC0DF83EDF0A9445145EFC03F83B0
:1059C00003250900FD14EFB06F8E6306850097B7BD
:1059D000010023A987CCF5F003250900EFB00F8D56
:1059E0006316850097B7010023AE87CA83A7090015
:1059F0000145850717B701002320F7CA97B70100B3
:105A000023A087CAEFC07FEA0325090097B70100EA
:105A100023A807C8EFB08F89E31F85F697B7010069
:105A200023A287C88DBFFD145145EFC04FFCADF4D4
:105A300061B74111114506C6EFB08F8197B50100DE
:105A4000938545A797B7010023A0A7C6EFB0AFEA9B
:105A500097B70100938747C59C43A5CF814801486C
:105A600097B70100938787C2094781461306004014
:105A700097B50100938505A517050000130545EFAF
:105A8000EFB0DF878148014897B701009387C7BF10
:105A9000054781461306004097B50100938505A38D
:105AA00017050000130505E3EFB05F85B24081489C
:105AB00001488147014781461306004097B5010020
:105AC000938545A117050000130525CE41016FB050
:105AD000FF82B2404101828097B701009387C7BB24
:105AE00097B60100938606BA984394426382E6060D
:105AF0009C4397B601009386A6B8944217B701005D
:105B00002322F7B897B701009387C7B898436382F9
:105B1000E6069C4397B60100938646B6944217B7B3
:105B20000100232FF7B497B70100938767B6984316
:105B30006382E6069C4317B701002321F7B497B7A9
:105B40000100938727B688437D153335A0008280F6
:105B5000854717B701002327F7B497B6010093864E
:105B600026B297B701009387E7B298439442E39235
:105B7000E6FA854717B701002326F7B297B601006A
:105B80009386C6AF97B70100938787B09843944236
:105B9000E392E6FA854717B701002325F7B097B7D8
:105BA0000100938727B088437D153335A00082809C
:105BB000B305B500930705006386B70003C7070068
:105BC000631607003385A74067800000938717009E
:105BD0006FF09FFE130101FB23229104232C41034C
:105BE0002322910323261104232481042320210549
:105BF000232E3103232A5103232861032326710313
:105C0000232481032320A103232EB101930C05003B
:105C1000138A05009304000063DE05003305A040ED
:105C20003337A000B305B040930C0500338AE5403C
:105C30009304F0FF63DA06003306C040B337C000B8
:105C4000B306D040B386F640930A06009389060057
:105C500013840C0013090A006396062817AB010091
:105C6000130B4B656370CA16B70701006372F61415
:105C70009307F00F63F4C70093098000B357360110
:105C8000330BFB0083470B0013050002B38737017A
:105C9000B309F540638C0900B3153A01B3D7FC0092
:105CA000B31A360133E9B70033943C0113DB0A0120
:105CB00093050B0013050900EF00507C130A050043
:105CC00093050B00939B0A0113050900EF009076E2
:105CD00093DB0B019305050013850B00EF00D072D9
:105CE000131A0A0193570401B367FA0063FAA70075
:105CF000B387570163E6570163F4A700B3875701E1
:105D00003389A74093050B0013050900EF001077B6
:105D1000130A050093050B0013050900EF009071AD
:105D20001314040193050500131A0A0113850B00CF
:105D300013540401EF00506D33648A00637AA400A9
:105D400033045401636654016374A40033045401A2
:105D50003304A4403354340193050000638A0400E3
:105D600033048040B3378000B305B040B385F540BD
:105D7000130504008320C104032481048324410407
:105D8000032901048329C103032A8103832A4103D0
:105D9000032B0103832BC102032C8102832C4102BC
:105DA000032D0102832DC10113010105678000004D
:105DB000B707000193090001E362F6EC9309800143
:105DC0006FF0DFEB631A0600930500001305100067
:105DD000EF005066930A0500B707010063FAFA0E58
:105DE0009307F00F63F4570193098000B3D73A018A
:105DF000330BFB0083470B001305000233095A41A4
:105E0000B3873701B309F540E38209EAB39A3A014F
:105E1000335BFA00B3153A01B3D7FC0093DB0A01F8
:105E200033E9B70013050B0093850B00EF001065F5
:105E3000130A050093850B00139C0A0113050B0040
:105E4000EF00505F135C0C019305050013050C0077
:105E5000EF00905B131A0A0193570901B367FA0028
:105E600033943C0163FAA700B387570163E65701F7
:105E700063F4A700B3875701338BA74093850B00CA
:105E800013050B00EF00905F130A050093850B00CC
:105E900013050B00EF00105A9305050013050C00C5
:105EA000EF00905693160901131A0A0193D60601C2
:105EB000B366DA0063FAA600B386560163E65601BC
:105EC00063F4A600B38656013389A6406FF01FDE47
:105ED000B707000193090001E3EAFAF09309800192
:105EE0006FF0DFF06376DA0093050A006FF01FE7CA
:105EF000B707010063FAF604930BF00F33B5DB002C
:105F00001315350033D7A60097A701009387873A6A
:105F1000B387E70083CB070093050002B38BAB0088
:105F2000338B7541631C0B0263E4460163EACC00CA
:105F30003384CC40B306DA4033B98C003389264130
:105F4000930509006FF09FE1B707000113050001F9
:105F5000E3EAF6FA130580016FF0DFFAB396660103
:105F6000335D7601336DDD00B35D7A01B3156A01EF
:105F700033DC7C0113540D01336CBC0013850D0020
:105F800093050400B3196601EF00504F930A050012
:105F90009305040013850D0033996C01931C0D01CA
:105FA000EF00504993DC0C01130A0500930505002E
:105FB00013850C00EF005045939A0A0113570C010A
:105FC00033E7EA00930D0A00637EA7003307A701B9
:105FD000930DFAFF6368A7016376A700930DEAFFAC
:105FE0003307A701330AA7409305040013050A00ED
:105FF000EF00D04893050400930A050013050A003A
:10600000EF005043930505001304050013850C00B1
:10601000EF00903F93150C01939A0A0193D5050167
:10602000B3E5BA001307040063FEA500B385A5011C
:106030001307F4FF63E8A50163F6A5001307E4FF67
:10604000B385A501939D0D01B70C0100B3EDED00E3
:106050001384FCFFB3F78D0033F48900338AA54025
:1060600013850700930504002326F10093DD0D013D
:10607000EF00903993050400930A050013850D0085
:10608000EF00903813DC090193050C002324A100D4
:1060900013850D00EF0050378327C10013040C0057
:1060A00093050400130C050013850700EF00D0359D
:1060B0008326810013D70A013305D5003307A700D3
:1060C0006374D700330C9C01B70701009387F7FF77
:1060D000935507013377F70013170701B3F7FA0059
:1060E000B3858501B307F7006366BA00631EBA0083
:1060F000637CF90033863741B3B7C700B385A54148
:10610000B385F54093070600B307F9403339F9002A
:10611000B305BA40B385254133947501B3D7670100
:106120003364F400B3D565016FF05FC3130101FD63
:1061300023229102232A51012326110223248102C2
:1061400023202103232E3101232C41012328610127
:106150002326710123248101232291012320A101FF
:10616000930A050093840500639E06381304060015
:106170009309050017A901001309C91363F8C51293
:10618000B7070100138B05006378F6101307F00FB3
:106190003337C70013173700B357E6003309F90048
:1061A000834609003387E60093060002B386E64083
:1061B000638C0600B394D40033D7EA003314D600BE
:1061C000336B9700B399DA00935A040193850A0060
:1061D00013050B00EF00902A1309050093850A00B0
:1061E000931B040113050B00EF00D02493DB0B017C
:1061F000930405009305050013850B00EF00D020E4
:106200001319090193D70901B367F900138A040030
:1062100063FEA700B3878700138AF4FF63E8870053
:1062200063F6A700138AE4FFB3878700B384A7400F
:1062300093850A0013850400EF005024130905001C
:1062400093850A0013850400EF00D01E939909017D
:1062500093040500930505001319090113850B002C
:1062600093D90901EF00501AB3693901138604006C
:1062700063FCA900B30934011386F4FF63E68900C7
:1062800063F4A9001386E4FF13140A013364C40005
:10629000130A00006F000013B70700011307000185
:1062A000E36CF6EE130780016FF01FEF138A060010
:1062B000631A06009305000013051000EF00901705
:1062C00013040500B7070100637EF4129307F00F73
:1062D00063F48700130A8000B35744013309F900BF
:1062E000034709009306000233074701B386E640DF
:1062F00063940612B3848440130A1000135B0401F4
:1063000093050B0013850400EF00501713090500D7
:1063100093050B0013850400931B0401EF009011FB
:1063200093DB0B01930405009305050013850B0017
:10633000EF00900D1319090193D70901B367F90014
:10634000938A040063FEA700B3878700938AF4FF53
:1063500063E8870063F6A700938AE4FFB3878700AA
:10636000B384A74093050B0013850400EF001011C0
:106370001309050093050B0013850400EF00900B33
:106380009399090193040500930505001319090168
:1063900013850B0093D90901EF001007B369390188
:1063A0001386040063FCA900B30934011386F4FFCB
:1063B00063E6890063F4A9001386E4FF13940A01DD
:1063C0003364C4001305040093050A008320C1024E
:1063D0000324810283244102032901028329C1018C
:1063E000032A8101832A4101032B0101832BC10070
:1063F000032C8100832C4100032D010013010103B4
:1064000067800000B7070001130A0001E366F4EC9F
:10641000130A80016FF05FEC3314D40033DAE40028
:10642000B399DA0033D7EA00935A0401B394D40045
:1064300093850A0013050A00336B9700EF001004E0
:106440001309050093850A0013050A00931B040134
:10645000EF00407E93DB0B019304050093050500DC
:1064600013850B00EF00407A1319090113570B0134
:106470003367E900138A0400637EA70033078700AF
:10648000138AF4FF636887006376A700138AE4FF2A
:1064900033078700B304A74093850A0013850400DF
:1064A000EF00C07D1309050093850A0013850400E1
:1064B000EF004078930405009305050013850B0059
:1064C000EF00807413170B0113570701131909010B
:1064D000B367E9001387040063FEA700B387870052
:1064E0001387F4FF63E8870063F6A7001387E4FFD0
:1064F000B3878700131A0A01B384A740336AEA00FE
:106500006FF0DFDF63ECD51EB707010063F4F6041C
:106510001307F00FB335D7009395350033D7B60086
:1065200097A70100938707D9B387E70003C7070040
:10653000130A00023307B700330AEA4063160A025F
:1065400013041000E3E096E833B6CA0013441600C3
:106550006FF05FE7B707000193050001E3E0F6FC89
:10656000930580016FF09FFBB35CE600B396460194
:10657000B3ECDC0033D4E40093DB0C01B3974401AB
:1065800033D7EA0093850B0013050400336BF70043
:10659000B3194601EF00806E1309050093850B00C7
:1065A00013050400139C0C01EF00C068135C0C0180
:1065B000930405009305050013050C00EF00C0646B
:1065C0001319090113570B013367E9001384040001
:1065D000637EA700330797011384F4FF6368970174
:1065E0006376A7001384E4FF33079701B304A74041
:1065F00093850B0013850400EF0040681309050024
:1066000093850B0013850400EF00C062930405001E
:106610009305050013050C00EF00005F93170B01B5
:106620001319090193D70701B367F9001386040012
:1066300063FEA700B38797011386F4FF63E8970111
:1066400063F6A7001386E4FFB387970113140401D0
:10665000B70B01003364C4001389FBFF337D2401B1
:1066600033F92901B384A7409305090013050D00F0
:10667000EF008059935C040193050900130B05009A
:1066800013850C00EF00405893D90901130C050045
:106690009385090013850C00EF00005713090500CE
:1066A0009385090013050D00EF00005633058501A1
:1066B00093570B013385A700637485013309790172
:1066C00093570501B387270163E6F402E392F4BC14
:1066D000B70701009387F7FF3375F5001315050120
:1066E000337BFB0033964A0133056501130A000032
:1066F000E37AA6CC1304F4FF6FF09FB9130A0000ED
:10670000130400006FF01FCC130101FB232481044C
:1067100023229104232E31032322910323261104E3
:1067200023202105232C4103232A5103232861031D
:1067300023267103232481032320A103232EB101E7
:10674000930C05009389050013040500938405004C
:10675000639E062613090600138A060097AA010005
:10676000938A4AB563F4C514B70701006376F6123D
:106770009307F00F63F4C700130A8000B357460174
:10678000B38AFA0003C70A00130500023307470162
:10679000330AE540630C0A00B395490133D7EC0096
:1067A00033194601B364B70033944C01935A09017D
:1067B00093850A0013850400EF00404C93090500FF
:1067C00093850A00131B090113850400EF0080461E
:1067D000135B0B019305050013050B00EF00C0428E
:1067E0009399090193570401B3E7F90063FAA700ED
:1067F000B387270163E6270163F4A700B387270166
:10680000B384A74093850A0013850400EF00004776
:106810009309050093850A0013850400EF00804169
:1068200013140401930505009399090113050B0046
:1068300013540401EF00403D33E48900637AA4005F
:1068400033042401636624016374A4003304240127
:106850003304A44033554401930500008320C10450
:106860000324810483244104032901048329C103EF
:10687000032A8103832A4103032B0103832BC102D3
:10688000032C8102832C4102032D0102832DC101BF
:106890001301010567800000B7070001130A00011A
:1068A000E36EF6EC130A80016FF05FED631A0600E9
:1068B0009305000013051000EF00C0371309050011
:1068C000B7070100637AF90E9307F00F63F427010D
:1068D000130A8000B3574901B38AFA0003C70A00BC
:1068E00013050002B384294133074701330AE54009
:1068F000E30E0AEA33194901B3DAE900B395490115
:1069000033D7EC0093540901336BB70013850A00A9
:1069100093850400EF0080369309050093850400F9
:10692000931B090113850A00EF00C03093DB0B01B4
:106930009305050013850B00EF00002D93990901C5
:1069400093570B01B3E7F90033944C0163FAA700A6
:10695000B387270163E6270163F4A700B387270104
:10696000B38AA7409385040013850A00EF00003125
:10697000930905009385040013850A00EF00802B1E
:106980009305050013850B00EF00002893150B01FC
:106990009399090193D50501B3E5B90063FAA50000
:1069A000B385250163E6250163F4A500B3852501C0
:1069B000B384A5406FF09FDFB7070001130A000101
:1069C000E36AF9F0130A80016FF0DFF0E3E8D5E83D
:1069D000B707010063FCF604930BF00F33B5DB003F
:1069E0001315350033D7A60097A701009387878C2E
:1069F000B387E70083CB070093050002B38BAB009E
:106A0000338B7541631E0B0263E4360163EACC00ED
:106A10003384CC40B386D94033B58C00B384A640D0
:106A200013050400938504006FF05FE3B7070001CE
:106A300013050001E3E8F6FA130580016FF09FFAF1
:106A4000B3966601335D7601336DDD0033D4790191
:106A5000B395690133DC7C0193540D01336CBC00A8
:106A60001305040093850400B31A6601EF000021AA
:106A7000130A0500938504001305040033996C0183
:106A8000931C0D01EF00001B93DC0C0113040500A7
:106A90009305050013850C00EF000017131A0A0177
:106AA00013570C013367EA00130A0400637EA70042
:106AB0003307A701130AF4FF6368A7016376A700F1
:106AC000130AE4FF3307A701B309A7409385040025
:106AD00013850900EF00801A938504001304050054
:106AE00013850900EF0000159305050093040500C8
:106AF00013850C00EF00401193150C0113140401D1
:106B000093D50501B365B4001387040063FEA500A7
:106B1000B385A5011387F4FF63E8A50163F6A5001B
:106B20001387E4FFB385A501131A0A01B70C01000E
:106B3000336AEA001384FCFFB3778A0033F48A00D7
:106B4000B384A54013850700930504002326F100B4
:106B5000135A0A01EF00400B930905009305040046
:106B600013050A00EF00400A13DC0A01930D05002B
:106B700093050C0013050A00EF0000098327C100EC
:106B8000130A050093050C0013850700EF00C007EA
:106B90003305B50113D709013307A7006374B701A3
:106BA000330A9A01B70701009387F7FF935507014E
:106BB0003377F70013170701B3F7F900B3854501E1
:106BC000B307F70063E6B400639EB400637CF9008A
:106BD00033865741B3B7C700B385A541B385F540A8
:106BE00093070600B307F9403339F900B385B44081
:106BF000B385254133947501B3D767013365F4003C
:106C0000B3D565016FF09FC513060500130500009D
:106C100093F61500638406003305C50093D515006F
:106C200013161600E39605FE678000006340050614
:106C300063C6050613860500930505001305F0FFDE
:106C4000630C060293061000637AB6006358C00016
:106C50001316160093961600E36AB6FE130500009D
:106C600063E6C500B385C5403365D50093D61600ED
:106C700013561600E39606FE67800000938200001C
:106C8000EFF05FFB13850500678002003305A0402D
:106C900063D80500B305B0406FF0DFF9B305B0402D
:106CA00093820000EFF01FF93305A04067800200D7
:106CB0009382000063CA0500634C0500EFF09FF764
:106CC0001385050067800200B305B040E35805FE58
:106CD0003305A040EFF01FF63305B0406780020097
:106CE000011122CC26CA2A84AE844AC84EC652C498
:106CF00056C206CEEFB04F8C1C4003290401B709E1
:106D00000001B3E59700930AC4000CC08144FD194B
:106D1000370A00021840638C2A03032609004A85BB
:106D2000B3654701B376360193175600758F032973
:106D3000490063C4070001E7F1BFE39DE6FC931738
:106D4000760063D30700D58CEFB0BFF4E1B793C4EE
:106D5000F4FFF98C04C0EFB02FAB0840F24062445E
:106D6000D2444249B249224A924A05618280411185
:106D700006C622C4EFE0AFE9EFE03F90EFE07FCB43
:106D800017E7FFFF1307070E8146054693054006E8
:106D9000179501001305056CEFC0BFC319C92A84FC
:106DA000EFB08F822A860147814685452285EFC054
:106DB000FFCEEFA05FD9B24022440145410182805D
:02000004800278
:100000005C45FEFF5A46FEFF6445FEFF5A46FEFF72
:100010005A46FEFF5A46FEFF5A46FEFF7C45FEFF4B
:100020005A46FEFF5A46FEFF9645FEFFA245FEFFDA
:100030005A46FEFFB445FEFFC045FEFFC045FEFF29
:10004000C045FEFFC045FEFFC045FEFFC045FEFFA8
:10005000C045FEFFC045FEFFC045FEFF5A46FEFFFD
:100060005A46FEFF5A46FEFF5A46FEFF5A46FEFF1C
:100070005A46FEFF5A46FEFF5A46FEFF5A46FEFF0C
:100080005A46FEFF5A46FEFF5A46FEFF5A46FEFFFC
:100090005A46FEFF5A46FEFF5A46FEFF5A46FEFFEC
:1000A0005A46FEFF5A46FEFF5A46FEFF5A46FEFFDC
:1000B0005A46FEFF5A46FEFF5A46FEFF5A46FEFFCC
:1000C0005A46FEFF5A46FEFF5A46FEFF5A46FEFFBC
:1000D0005A46FEFF5A46FEFF5A46FEFF5A46FEFFAC
:1000E0005A46FEFF5A46FEFF5A46FEFF5A46FEFF9C
:1000F0005A46FEFF5A46FEFF5A46FEFF5A46FEFF8C
:10010000F445FEFF0A46FEFF5A46FEFF5A46FEFF32
:100110005A46FEFF5A46FEFF5A46FEFF5A46FEFF6B
:100120005A46FEFF5046FEFF5A46FEFF5A46FEFF65
:100130000244FEFFBA44FEFF5A46FEFF5A46FEFF47
:10014000F044FEFF5A46FEFF4845FEFF5A46FEFFBA
:100150005A46FEFF7645FEFF6849FEFFBC49FEFF9A
:100160007049FEFFBC49FEFFBC49FEFFBC49FEFFD3
:10017000BC49FEFF6248FEFFBC49FEFFBC49FEFFD2
:100180007C48FEFF8848FEFFBC49FEFF9A48FEFF00
:10019000A648FEFFA648FEFFA648FEFFA648FEFFB3
:1001A000A648FEFFA648FEFFA648FEFFA648FEFFA3
:1001B000A648FEFFBC49FEFFBC49FEFFBC49FEFF4E
:1001C000BC49FEFFBC49FEFFBC49FEFFBC49FEFF27
:1001D000BC49FEFFBC49FEFFBC49FEFFBC49FEFF17
:1001E000BC49FEFFBC49FEFFBC49FEFFBC49FEFF07
:1001F000BC49FEFFBC49FEFFBC49FEFFBC49FEFFF7
:10020000BC49FEFFBC49FEFFBC49FEFFBC49FEFFE6
:10021000BC49FEFFBC49FEFFBC49FEFFBC49FEFFD6
:10022000BC49FEFFBC49FEFFBC49FEFFBC49FEFFC6
:10023000BC49FEFFBC49FEFFBC49FEFFBC49FEFFB6
:10024000BC49FEFFBC49FEFFBC49FEFFBC49FEFFA6
:10025000BC49FEFFBC49FEFFDA48FEFF0849FEFF2D
:10026000BC49FEFFBC49FEFFBC49FEFFBC49FEFF86
:10027000BC49FEFFBC49FEFFBC49FEFF5E49FEFFD4
:10028000BC49FEFFBC49FEFFC046FEFFBA47FEFF69
:10029000BC49FEFFBC49FEFF2C48FEFFBC49FEFFE7
:1002A0005248FEFFBC49FEFFBC49FEFFB649FEFFB7
:1002B000000102020303030304040404040404040D
:1002C00005050505050505050505050505050505DE
:1002D00006060606060606060606060606060606BE
:1002E00006060606060606060606060606060606AE
:1002F000070707070707070707070707070707078E
:10030000070707070707070707070707070707077D
:10031000070707070707070707070707070707076D
:10032000070707070707070707070707070707075D
:10033000080808080808080808080808080808083D
:10034000080808080808080808080808080808082D
:10035000080808080808080808080808080808081D
:10036000080808080808080808080808080808080D
:1003700008080808080808080808080808080808FD
:1003800008080808080808080808080808080808ED
:1003900008080808080808080808080808080808DD
:1003A00008080808080808080808080808080808CD
:1003B000546D725100000000546D7220537663003A
:1003C000286E756C6C2900004572726F7220696E20
:1003D00020626C6F636B2074696D65207465737443
:1003E000207461736B73200D0A0000004572726FF8
:1003F0007220696E20636F756E74696E6720736515
:100400006D6170686F7265207461736B73200D0A83
:10041000000000004572726F7220696E2072656381
:10042000757273697665206D757465782074617373
:100430006B73200D0A0000006D69616F750A000082
:100440006D69616F75320A0068756E6772790A00AE
:10045000436865636B54696D65720000426C6F633D
:100460006B5F54696D655F517565756500000000CF
:100470004254657374310000425465737432000055
:10048000436F756E74696E675F53656D5F31000011
:10049000436F756E74696E675F53656D5F32000000
:1004A000434E543100000000434E5432000000001F
:1004B0005265637572736976655F4D757465780012
:1004C0005265633100000000526563320000000095
:0804D0005265633300000000D7
:1004D8001000000000000000017A5200017C0101B8
:1004E8001B0D02005000000018000000E056FEFF3F
:1004F8005805000000440E507489039406990B8136
:1005080001880292049305950796089709980A9A14
:100518000C9B0D036C010AC144C844C944D244D39E
:1005280044D444D544D644D744D844D944DA44DBE7
:10053800440E00440B0000004C0000006C0000005A
:10054800E45BFEFFDC05000000440E307089039573
:1005580007810188029204930594069608970998E2
:100568000A990B9A0C0370020AC144C844C944D2C0
:1005780044D344D444D544D644D744D844D944DA9F
:10058800440E00440B00000050000000BC000000B6
:100598007061FEFF0005000000440E507488028957
:1005A800039305990B810192049406950796089781
:1005B80009980A9A0C9B0D0320010AC144C844C932
:1005C80044D244D344D444D544D644D744D844D957
:0C05D80044DA44DB440E00440B00000039
:0806A800FC8F010004000000BA
:040000058000004037
:00000001FF
